:020000040000FA
:10000000007D0400010000002A430000DE410000E2
:1000100014420000EC420000124300002A4300009A
:100020002A4300002A4300002A4300002A4300001C
:100030002A430000024400002A4300002A43000033
:100040002A4300007045000066470000D83C0000CD
:100050002A4300002A4300002A4300002A430000EC
:100060002A4300002A4300002A4300002A430000DC
:100070002A4300002A4300002A4300002A430000CC
:100080002A4300002A430000BE5800002A43000013
:100090002A4300002A4300002A4300002A430000AC
:1000A0002A4300002A4300002A4300002A4300009C
:1000B0002A4300002A430000E43F0000583F0000AC
:1000C0002A4300002A4300002A4300002A4300007C
:1000D0002A4300002A4300002A4300002A4300006C
:1000E0002A4300002A4300002A4300002A4300005C
:1000F0002A4300002A4300002A4300002A4300004C
:1001000000000000000000002A430000DE41000063
:1001100014420000EC420000124300002A43000099
:100120002A4300002A4300002A4300002A4300001B
:100130002A430000024400002A4300002A43000032
:100140002A4300007045000066470000D83C0000CC
:100150002A4300002A4300002A4300002A430000EB
:100160002A4300002A4300002A4300002A430000DB
:100170002A4300002A4300002A4300002A430000CB
:100180002A4300002A430000BE5800002A43000012
:100190002A4300002A4300002A4300002A430000AB
:1001A0002A4300002A4300002A4300002A4300009B
:1001B0002A4300002A430000E43F0000583F0000AB
:1001C0002A4300002A4300002A4300002A4300007B
:1001D0002A4300002A4300002A4300002A4300006B
:1001E0002A4300002A4300002A4300002A4300005B
:1001F0002A4300002A4300002A4300002A4300004B
:10020000140104000000000094010400000000003C
:10021000C2010400000000000E0B040000000000FA
:1002200000000400000000000F1721008079220068
:100230000001880000000000050007000C00070016
:10024000BC260200000000000040DA000000FE00B2
:100250004440A90000A521000000E0000300320096
:1002600000002000A00188004440A8000000060013
:10027000E07E2600010020001600370062004000EA
:10028000E0804800910188009001BA0062004000BF
:10029000E0804800910188009002BA0062004000AE
:1002A000E08048000002EB006028E10005003A0011
:1002B0008301E90007003300038009000059EB00C7
:1002C000040037006128E100010032000082EB00E9
:1002D00005000700910188001001BA000200E0004B
:1002E000E6FF3A00000005009101880080027800D6
:1002F00062004000E08048003559BA008301E900FF
:10030000080032002559BA008301E90005003200D7
:100310000400E000F4FF320015D9BA008301E900BF
:10032000F1FF3A0000000600881F78000204780000
:1003300082000700080040004F047800000006001B
:100340000000FA00881F7800000478003FB9970089
:10035000EA81570080007800401920007E000700E5
:10036000800078000000E000020035000040EB0053
:1003700000F47800010078004F0478000080FA0053
:1003800000000600889FBE0080047800010078000D
:100390000204780089017800110020000F00070096
:1003A00089007800880F5000010032008000EB00C7
:1003B000010078004F04BE00000006000000FA00B3
:1003C0004FB99700E8815700C1BE2000201C2000D3
:1003D000610007000080FA0000000600E487470083
:1003E000889FBE008A9FBE008C9FBE008E1F780033
:1003F00081BF9F00820078008304780000077800A6
:100400000FB997000116B8008C0578000001EB00C9
:100410000C00E00042003200010178008FB9970023
:100420000300E0003E0032000C00E0002E0032002D
:10043000C900900069009000808F500004003900CE
:1004400009007800F90007000000E00026003500F0
:1004500019A8A300060032000B017800A1002000BB
:100460000E00780036010700000578000100370013
:100470000005EB000B0478000A00E00002003200E7
:100480000E0055000004E80069009000C9019000CA
:1004900003005000880F5000020031000005EB00FF
:1004A00000047800080178008E00780003007800CE
:1004B0002200070008074700888555004900900082
:1004C00008004000C00498000A00E0000400320068
:1004D00009007800230107000000E00002003A0054
:1004E0000B00E000D2FF3A0019B8A300020032006E
:1004F000090078001B01070000C0200019006000FF
:100500000200320049009000E00498000B00560001
:100510008FB99700110009000380D800000178000E
:10052000020078004F0778004F06BE004F05BE005E
:100530004F04BE004F00B1000000060080017800AB
:100540000200E00003003200B15978000201E90026
:10055000FDFF3A00000006006200FA00889FBE001E
:100560008A9FBE000004BE00020578008300780068
:100570006A80570037010700F88F9F0089979F0016
:100580000000EB00909F9F001A80FB008005FB009D
:100590000000EA00CF04DE000904780050022000C9
:1005A000808F550001003A000904E9000800E000CE
:1005B0000C0034000F909700080178008A00780042
:1005C000FF8997000300010080979F008080EB0067
:1005D0000000E000900032001F98970008004000E3
:1005E000909F9F000905450050022000808F550014
:1005F000040032000B00E000E3FF3A009F989700F0
:10060000850037000000EB00F0979F00E0979F0007
:10061000D0979F00C0979F00B0979F00A0979F0022
:10062000B09F9F000900370060D02000008050007C
:100630000000D000C1D0200001004000BF9897000A
:1006400090807000B19F9F000A05E8009A00FB00AF
:1006500060D0200001010700800078000000E00069
:10066000F1FF3A00A0C2B3009A4F10000E003A000A
:100670003FB897000080E900B0BF9F0010007800ED
:10068000A09F9F000000E00005003D000000EA0080
:10069000A09F9F003F9897000020A000B09F9F0060
:1006A0000A05E80011003700A19F9F000B003700EA
:1006B000AF989700F0FF2700808F500006003200AF
:1006C0006A09B9001A00FB000200400001FD2F007A
:1006D00001004000A09F9F000A05E8001A00FB00EF
:1006E000E60007000000E000F1FF3A00E0C2B300BE
:1006F0009A4F1000030032000080EB00809F9F00A3
:100700001C003700A0C2B300DA4F100007003A0007
:100710003FB897000080E900B0BF9F00100078004C
:10072000809F9F000A05E800120037000000EB00E0
:10073000809F9F000B0037008F989700F0FF2700E5
:10074000808F5000060032006A09B9001A00FB00D1
:100750000200400001FD2F0001004000809F9F002B
:100760000A05E8001A00FB00C40007000000E000D2
:10077000F1FF3A009A00FB00E0D72000B700070025
:100780008040EB000000E00001003200BA40780039
:10079000817F9F0080C6B30080CF500004003A00E4
:1007A0009ACF100002003A00664050000700370060
:1007B0008F789700C0C6B30080CF500005003A0084
:1007C0009ACF100003003A0065404000807F9F00F0
:1007D0000A05E800A0FB2F00008447003A4178009A
:1007E00088017800EA80570060F92F000F00400070
:1007F000760107000000E00006003A00880078005B
:1008000060F92F000F004000A20007000000E00088
:100810005DFF3D008080EB00010078004F05BE00C9
:100820004F04BE000080FA0000000600889FBE0052
:1008300000047800C0019000600090008000EB0090
:10084000808F51003B0039001801780020002900FA
:1008500000006100E20F5000090032000200780041
:100860000090A0000200E0000200350000202400FB
:1008700000007100000C78008080EB002D00370034
:100880000100260001006100810F500008003A00BD
:1008900038009000808F5100050039000800780072
:1008A000300007008080EB000000E00021003A00EB
:1008B00000C020001800600017003A00600220000D
:1008C00008004000A8049000808F540012003A00F5
:1008D00000202000260307008000780020049800F4
:1008E0000000E00005003A0029049800490498003F
:1008F0000900E80030049800060037001860A000E6
:10090000400498000020B00030049800410C98008A
:10091000510C98004D0307002800900050049800E7
:10092000380090006004980000002600180C700049
:100930008000EB00010078004F04BE0000000600BC
:100940000200E0000500320090CF100004003200E9
:100950000000E8000201E900FBFF3A000000EB00A4
:1009600000000600889FBE00000478000000E00040
:100970000F003A006044B8000800D000C1C3200056
:10098000608078000000E00004003200F5FF0700FE
:100990000000E00001003D008084EB000804E80056
:1009A00009007800E70F540028003C00F2FF3700F0
:1009B00010D8A30024003200A00490004000900052
:1009C000808F54000B003100090150003840900026
:1009D0000000FB0089007800050907000000E00026
:1009E000110034008084440048009000808F54003F
:1009F000F5FF390028009000400498009800780026
:100A000000C020000080600002003200A8049000B6
:100A100001003700B804900001E8A300090032008B
:100A20006904980008003700A8009000410498006D
:100A300061049800510C98001890A0000080EB0011
:100A400002003700590C98000000EB004F04BE0074
:100A500000000600010878000000060090CF10009A
:100A6000050032001004E00001003A00000005001B
:100A7000D0CF1000FBFF3A00000006000003B100D9
:100A8000030035009000B10001003C00100005009B
:100A9000000005000400FA00889FBE008A9FBE0087
:100AA0008C1F780000047800010678007008900020
:100AB000F8009000010050008808900001005000EC
:100AC0009808900001005000A80890000100500014
:100AD000B808900001005000C8089000810550003F
:100AE0000002220090BF9F0000032300A0BF9F00D0
:100AF000081090000028A30018003A000B00E00046
:100B0000160034000B0578008A047800E20F5500C7
:100B100001003600290020000900E0000C0034002C
:100B200058009000C801900009017800EE8057003D
:100B300003000100500498008080EB000000E000FA
:100B40009C0032006808900009004000600C98008A
:100B5000090555004240A900EBFF3C0078019000D8
:100B60000200E0000C00340058009000C801900022
:100B70008C00780003000100500498008080EB0096
:100B80000000E0008B00320068089000F800900040
:100B900001004000600C9800080890000000E00090
:100BA00016003400000578008A047800E20F550032
:100BB00001003600290020000900E0000C0034008C
:100BC00058009000C801900009017800EC8057009F
:100BD00003000100500498008080EB000000E0005A
:100BE000740032006808900009004000600C980012
:100BF000090555004240A900EBFF3C001809900090
:100C00000200E0000C003400E80090005800900062
:100C1000C801900003000100500498008080EB00A0
:100C20000000E0006300320068089000980890001F
:100C300001004000600C9800280890000000E000CF
:100C400016003400000578008A047800E20F550091
:100C500001003600290020000900E0000C003400EB
:100C600058009000C801900009017800EC805700FE
:100C700003000100500498008080EB000000E000B9
:100C80004C0032006808900009004000600C980099
:100C9000090555004240A900EBFF3C0038099000CF
:100CA0000200E0000E003400E800900018089000F8
:100CB0008080400058009000C801900003000100AF
:100CC000500498008080EB000000E0003900320002
:100CD00068089000B808900001004000600C98007F
:100CE000480890000000E00016003400000578007D
:100CF0008A047800E20F5500010036002900200028
:100D00000900E0000C00340058009000C801900079
:100D100009017800EC80570003000100500498009E
:100D20008080EB000000E0002200320068089000A4
:100D300009004000600C9800090555004240A900D8
:100D4000EBFF3C00081090000028A30018003200C0
:100D50000B00E000160034000B0578008A047800D0
:100D6000E20F550001003600290020000900E000D4
:100D70000C00340058009000C80190000901780070
:100D8000EE80570003000100500498008080EB00C3
:100D90000000E000070032006808900009004000F1
:100DA000600C9800090555004240A900EBFF3C008B
:100DB0008000EB00010078004F0678004F05BE0070
:100DC0004F04BE000080FA0000000600889FBE00AD
:100DD0008A1F78000004780001027800024578003C
:100DE000830478000200FB00CF80DE005002B100D7
:100DF0000180B10032052000820F5000E08F5800C2
:100E000095013E00006001008D013700920137001E
:100E100091013700900137008F0137008E013700B4
:100E20008D0137008C0137008B0137008A013700B4
:100E300089013700880137008701370086013700B4
:100E400085013700840137008301370082013700B4
:100E500081013700800137007F0137007E013700B4
:100E60007D0137007C0137007B0137007A013700B4
:100E70007901370078013700ED003700760137003F
:100E80007501370074013700E9003700E8003700CA
:100E9000E7003700700137006F0137006E0137003F
:100EA0006D0137006C0137006B0137006A013700B4
:100EB00069013700680137006701370066013700B4
:100EC0004B013700640137006301370062013700CE
:100ED00061013700800037005F0137005E01370095
:100EE0005D0137005C0137005B0137005A013700B4
:100EF0005901370058013700CD003700560137003F
:100F0000150037001C003700C9003700C800370043
:100F1000C700370050013700170037004E01370077
:100F20004D0137004C0137004B013700EC00370012
:100F3000690037001F0137004701370046013700BD
:100F40002B013700440137006300370042013700AE
:100F500041013700600037006E0144001200780044
:100F6000808141009480E900010A78000009E800CE
:100F70009149780041013700A8609000C0C6B300D5
:100F800080CF50000A003A0094007800648050003E
:100F9000000A78001000BE004F89DE00CF91DE000D
:100FA0000002BE00020378008203780015003700BB
:100FB00010C7B30080CF500002003A00140178003F
:100FC0000400370014017800A0C6B30080CF5000A1
:100FD00005003A0068005100000A78003002BE00A7
:100FE0002003BE00070037000280E900000A7800F5
:100FF0001000780000027800CFA2DE000503780020
:1010000086037800049CBE000694BE00A860900091
:1010100080C6B30080CF50000F00320020C6B3005E
:1010200080CF500006003A00184078000000FB0016
:10103000CF80DE0001017800820178000A003700CD
:1010400040C7B30080CF500003003200664040002C
:1010500080CF500006003A0018007800CF80DE00F4
:101060000101780082017800009CBE000294BE005D
:101070003800BE002801BE00E00F5000E08F58008D
:10108000E00F5900E08F590004003D006E0144005C
:1010900092007800D0C2B3000C0037000810900016
:1010A0000018A300040032006E0144009200780092
:1010B000B0C2B300050037000008A300570032009B
:1010C0006E0144009200780000C2B30080F4780002
:1010D0000109E80051003700A8609000C0C6B300C5
:1010E00080CF500006003A009400780064805000E1
:1010F000000A78001002BE006033B8001500370007
:1011000010C7B30080CF500002003A0014017800ED
:101110000400370014017800A0C6B30080CF50004F
:1011200005003A0068005100000A78003002BE0055
:101130002003BE00070037000280E900000A7800A3
:101140001000780000027800050020000600200052
:1011500007002000049CBE000694BE00A86090001A
:1011600080C6B30080CF50000F00320020C6B3000D
:1011700080CF500006003A00184078000080FB0045
:101180000100200002002000030020000A003700B8
:1011900040C7B30080CF50000300320066404000DB
:1011A00080CF500006003A001800780001002000AF
:1011B0000200200003002000009CBE000294BE003C
:1011C000081090000038A300140032003800BE0060
:1011D0002801BE00E00F5000E08F5800E00F5900DA
:1011E000E08F59000D00320080C7B300804F5500DA
:1011F0000300320080C5B300804F550007003A005D
:101200006E0044009000780002C3B30082F47800BE
:101210008100E8008AF478000108E8007800900076
:1012200000804400600498008A4078006D00370018
:10123000A860900014017800C0C4B30080CF5000B3
:1012400005003A0068005100000A78005001BE0015
:101250004000BE000400370064005100000A78001E
:101260001000BE00B4070700009CBE000294BE0040
:10127000380090000000E00004003D006E014400D2
:1012800092007800D0C2B3000C0037000810900024
:101290000018A300040032006E01440092007800A0
:1012A000B0C2B300050037000008A30005003200FB
:1012B0006E0144009200780000C2B30080F4780010
:1012C0000109E80078009000008044006004980064
:1012D0008A40780008007800D901070067003700CD
:1012E000286090008000FB00C0062000808F500026
:1012F000230032000A003C0064005000808F500040
:101300002600320004003C0066005000808F500030
:101310000B00320021003700A00620000500370036
:1013200040072000808F50001C0032001B003C0052
:1013300063005000808F5000070032001700370014
:101340001480E900000A780010007800485C9000E2
:1013500008487800490037001480E900000A780046
:101360001002780068089000CF80DE00010178004C
:1013700082017800009ABE000292BE003F00370052
:101380001480E900000A78001001780068089000D5
:10139000CF80DE000089BE00380037001480E900ED
:1013A000000A780010007800680C900008087800A7
:1013B000320037001480E900000A7800100078003D
:1013C000CF80DE000101780082017800009CBE0021
:1013D0000294BE00780090000080440060049800F1
:1013E00081C7B30008007800DC0007002300370045
:1013F0001480E900000A780010007800600498006A
:10140000580990000200E00002003D00850107003D
:10141000090037008000EB0049FD070080007800DC
:101420000000E000030032006800900000805000DF
:101430000100370058089000100C98000F0037008A
:101440006E0144009200780050C2B30080F1780031
:101450000109E80009003700EE004400110078009F
:10146000808144000A4278008008E8000A04E00015
:1014700001003A0054C2B300844978000000EB0038
:101480004F0578004F04BE0000000600889FBE0094
:101490008004780051698000010078000100E000BC
:1014A0000A003A00C1D220002C0DE2001C003200DC
:1014B00011007800908F5400140036008080E800FE
:1014C0001100E000FAFF3A00150037001100E000BB
:1014D0000600320011017800928F54000B00360094
:1014E0008280E8001100E000FAFF3A001001780065
:1014F000C1D2200060698000820F500008003200D5
:1015000011007800908F540002003E000100780026
:10151000150037008080E800910F1100F8FF3A00B5
:1015200078698000890F54000100310009047800B7
:101530000800780099030700000178000000E0002F
:1015400005003A000000EB00890F5400060032004D
:101550000804D100F3FF3700081978000200780072
:1015600095030700CBFF37004F04BE0000000600C4
:10157000881F7800630440000800A1000001EB0010
:10158000800F540022003600E30F540001003E009B
:101590004800200008007800BCFF070080007800A9
:1015A0000001EB000000E00019003200100178009B
:1015B0009201780064805100880F500003003100D0
:1015C00012009000800878000700370008004100F2
:1015D0008008780012029000140098001100780032
:1015E0000888510008097800910078000100E000A7
:1015F00004003200110090008180E8000000E0004B
:1016000001003A008000EB00516988000281E80087
:10161000020078004F04780000000600881F780060
:10162000880020000800D000C1C32000608078003E
:101630000000E000010032000A0007000804E90091
:10164000F8FF3700E0B0200094033700424DE2007D
:1016500003003A00FBFF070020C0B30042EDB700D3
:1016600000000600889FBE0000047800BDFC070053
:10167000800478001868A30002003200280090005F
:101680004D0307000000EB00200498003840900054
:101690000004E000050035000000FB000206070022
:1016A0000000E000010032008084EB001810900080
:1016B0000000E00008003200040607000000E0001F
:1016C000010032008084EB00181090003A030700FC
:1016D0000000EB00101498001878A3000E003200F0
:1016E0008000EB000100D000C2C3200002004000D7
:1016F000900F1400060032008100E800E78F5000D0
:10170000F8FF3600080078002B03070010003700B0
:101710000008EB00FBFF3700000CEB0000C0EB0003
:101720003044980060022000080040002004980027
:101730004004980050049800400C98006004980001
:10174000500C98007004980076004400000C98003B
:10175000090078004F04BE00000006006F02B000D0
:10176000889FBE008A9FBE008C9FBE008E1F78009F
:101770008006780050CA2000B0B79F0080C5B30033
:1017800080CF50000200320042C92000B2B79F0053
:1017900083002000C3B79F00F0C6B30080CF500085
:1017A0000A0032006940400080CF5000050032003E
:1017B000A4002000C4B79F0080C5B30080CF5000B4
:1017C00002003A0000012000C0B79F008E012000F7
:1017D0003D04BE002D05BE0040C6B30080CF5000C2
:1017E000030032006540400080CF50000A003A00FC
:1017F000E00F5400E08F5C00E00F5D00E08F5D00C3
:1018000005003D000800BE000A01BE0045060700B5
:101810000205BE000004BE00E00F5400E08F5C0033
:10182000E00F5D00E08F5D0003003A005D0890006E
:101830000000E0000C0032007E012000CFB09700D5
:1018400001027800CFA2DE0005037800860378004D
:101850000800BE000A01BE00E70607003FB297007D
:1018600064407800D0E79F004FB09700CF80DE0043
:101870000101780082017800D0B79F00E1B79F0096
:10188000F2B79F0083BF9F000203BE000002BE00AC
:101890000800BE000A01BE00D0060700809EBE0000
:1018A0008296BE00E00F5000E08F5800E00F590014
:1018B000E08F5900220034000E00E00020003400C8
:1018C0003D00BE002D01BE005FB29700EFB2970051
:1018D0007FB397008FBB9700CB0607000205BE00C1
:1018E0000004BE000E07E900E1FC2F008F804000DD
:1018F000010647005FB29700EFB297007FB39700F1
:101900008FBB97000800BE000A01BE00CD0507008E
:101910001D0010003FB19700624E7800889EBE0007
:101920008A96BE00E00F5400E08F5C00E00F5D007F
:10193000E08F5D00020034000E00E000E0FF3C009C
:10194000CFB19700E88F510010003A000D109000C1
:101950000038A3000D003200F70F570006003E00CC
:10196000E4FC2F000E024200E4C07F0000C3B3007D
:1019700080CF5000050032000E07E90000C3B3001D
:10198000E1FC2F008E80400080F07F00780117007E
:10199000920E98006D009000E3FC2F008F814100B3
:1019A0008E804100E5FA07001D0E90005D08900052
:1019B000800F560006003D000C005000800E98007D
:1019C0000D1090000040A100801698000F00370015
:1019D0000000E0000D003D000D109000740060005C
:1019E000F00F500009003A007D089000FD009000C3
:1019F000010050008D089000010050000C075000BD
:101A00004240A900010034008E0E98004F07780074
:101A10004F06BE004F05BE004F04BE006F02B1006E
:101A200000000600800078001004E0000200320090
:101A30005104E000FEFF3A00008050000000060064
:101A4000EF04B000889FBE008A9FBE008C9FBE003E
:101A50008E1F7800C0AF9F00A1DF9F0060FA2F00AB
:101A60000F004000E0AF9F00CFAA97005503BE00D3
:101A70004502BE0084AF9F0095AF9F00A6AF9F00B8
:101A8000B7AF9F0010C6B30080CF500016003200E1
:101A900010C4B30080CF5000130032004FAB97004A
:101AA000560890000000E00003003D0060002000A8
:101AB000500B98000C0037000000E0000A003A00CC
:101AC00070C6B300AFDB970080CF53000300320035
:101AD00070C4B30080CF530003003A001000200010
:101AE000CFA89700D0089800CFA89700E2FC2F005D
:101AF000028047007602070080017800E20F500064
:101B000014003A00CFA99700E300900030002000B5
:101B10009009980010C6B3002FDA9700804F52004A
:101B20000A00320064404000804F5200070032003B
:101B30000040E800804F520004003200C2D4200070
:101B40000040E800804F520017003A0002D5200004
:101B5000150037000000E00018003400CFAA9700FD
:101B6000E500900030002000900A980010C6B300F5
:101B70002FDB9700804F53000A0032006440400082
:101B8000804F5300070032000040E800804F5300B0
:101B90000400320042D520000040E800804F53008E
:101BA00001003A0082D52000B25878000200780087
:101BB000B058780090487800F201370014C6B3009E
:101BC000AFDB970084CF53000300320010C4B30092
:101BD00080CF530010003A004FA89700EC0040005F
:101BE0001101780000C3B300005978008208E800B2
:101BF00080C7B300AFD8970084CF500001003200F7
:101C000080C5B300004978004FA99700720090008A
:101C10000080E800700198000300E00003003A0033
:101C20008006EB00FDA79F00D001370011C6B3006E
:101C3000AFD9970081CF51000300320010C4B30028
:101C400080CF5100AD003A00CED520002FDA9700AA
:101C5000814F520001003200DED62000CFAA97004B
:101C6000550890008006E8000000E00001003D00FB
:101C70001D0220000D06E8004FAB97003604BE00A1
:101C80002605BE006022B8006033B8000FA8970098
:101C90009FA897002FA99700BFA997005606070095
:101CA0000000E00001003D000BF0A20088AF9F00A3
:101CB00099AF9F00AAAF9F00BBAF9F007FA0970086
:101CC00064005000F0A79F00EFAB9700805BEB0033
:101CD000E7AF9F003F003700C20120000300200053
:101CE00001FD2F0001804700270207000FAA97007F
:101CF0009FAA97002FAB9700BFAB9700F4AF9F0050
:101D000085B79F0096B79F00A7B79F000400BE004D
:101D10000601BE003D0607000004BE000005BE002F
:101D2000670656004240A9000C0034006306070015
:101D30000002BE000203BE007FA897008FB097008C
:101D40001FB19700AFB197005F06070080AF9F00FB
:101D500091AF9F00A2AF9F00B3AF9F00EFAA970083
:101D6000E7824200E5AF9F0070002000E00F5400C2
:101D7000E08F5C000D003400600020006FAB970026
:101D80006F636500E6AF9F00CC5BDD004455DE006D
:101D90000A857300C4DDDE00E00F5500E08F5D00B2
:101DA000020034000000E900F4FF3B000000E900FD
:101DB00005003300EFA897008060EB00E1AF9F00C3
:101DC0000000E900FBFF3B006FA99700670141009D
:101DD000E2AF9F000C00E000090034006022B80070
:101DE0006033B8000FA897009FA897002FA997000D
:101DF000BFA99700360607000000E000B6FF3C00D0
:101E0000EFA9970064FA2F000F02420004805100EE
:101E10000006E90075FA2F0085824700E5AF9F00B4
:101E20008D0F560001003D008C0678000D00E0008B
:101E30002B0035008C8F560005003D006FAB9700DE
:101E400066C07E00F2C0B300E74F500001003C00C6
:101E50000041EB008D00E900EFAB970067C0780010
:101E6000824F500006003A008D06E9008100E9002B
:101E7000EFA9970063C07800824F5000FAFF32004C
:101E8000EF4F510004003A006FAA970064C0780039
:101E90000040E80000F278000100E00007003D008B
:101EA000EFAA97008502E900E5AF9F008D06E800E4
:101EB0007FA0970064004000F0A79F008D00E9001C
:101EC000070033006FAB970066C078000000FB008E
:101ED0006E40780000F378008100E900F9FF3B00D4
:101EE000CFAB9700570890000000E0001F013D00B5
:101EF0000D00E900D00B98001C0137000FAC9700D3
:101F00009FAC97002FAD9700BFAD97006022B8003F
:101F10006033B8000800BE000A01BE00B605070025
:101F20000000E00005003D000BF0A20088AF9F001C
:101F300099AF9F00AAAF9F00BBAF9F007FA0970003
:101F4000725927000280B900026A2800130020009D
:101F50000C040700E4005000F1A79F001D003B00A7
:101F600063801000C1FF2F00010460000800EA0038
:101F7000F0A79F008004EB000800E0004700340059
:101F80000808A3000E0032006848B800C2C4200050
:101F9000020040003002BE002003BE000FA89700E0
:101FA0009FA897002FA99700BFA99700CD0507000C
:101FB00080AF9F0091AF9F00A2AF9F00B3AF9F0083
:101FC0000884D1008904E8000800E000ECFF3C0030
:101FD000320037000100E000300034006022B80019
:101FE0000600200007FF2300B4B79F00C5B79F007D
:101FF000D6B79F00E7B79F00C0FF2F0000806000AA
:10200000F0A79F00000478008004EB001600340065
:102010000808A300100032006848B800C5C42000BA
:10202000050040003002BE002003BE003FB0970014
:10203000CFB097005FB19700EFB19700A9050700F7
:102040000002BE000203BE00B4B79F00C5B79F00E8
:10205000D6B79F00E7B79F000884D1008904E80045
:102060000800E000EAFF3C003FB29700CFB29700C3
:102070005FB39700EFB397000FA897009FA8970052
:102080002FA99700BFA997000B06070080AF9F00FC
:1020900091AF9F00A2AF9F00B3AF9F004FAB9700DF
:1020A000D608900060C6B300AFDB970080CF530026
:1020B000040032006687400060C4B30080CF530044
:1020C00003003A007FA09700008040006A074000AC
:1020D000F30F5700010034003E01200000C3B3009D
:1020E000EFA8970080587800E1AF9F003A003700D2
:1020F0000800BE000A01BE00440507000006BE003D
:10210000F0B79F0081BF9F00680757004240A900B9
:102110000E003400690507000002BE000203BE0085
:102120000800BE000A01BE00670507006022B80073
:1021300046782D00771924006A05070080AF9F00BC
:1021400091AF9F00A2AF9F00B3AF9F00EFA9970090
:10215000E8814100E3AF9F0088002000E00F5600B7
:10216000E08F5E001100340078002000A200200003
:10217000030020007FB097008FB897007801070018
:102180006FAA970005C3B30005624100E4AF9F004A
:10219000F0B79F0081BF9F00E00F5000E08F580014
:1021A000020034000804E900F0FF3B000804E900E5
:1021B0000600330000C3B300EFAB970080637800E4
:1021C000E7AF9F000804E900FAFF3B006FA8970003
:1021D00068004000E0AF9F000E00E0000B003400FC
:1021E0000FAC97009FAC97002FAD9700BFAD970045
:1021F0006022B8006033B8000800BE000A01BE00CB
:10220000330507000000E000B9FF3C00EFA897008D
:1022100062FA2F000F014100028050000007E90020
:1022200073FA2F0083814700E3AF9F007FA09700E0
:1022300067004000F0A79F0001C3B30093CF1000D8
:102240000A003A000E07E9007FA097000000E900AD
:10225000F0A79F006FAA97000402E800E4AF9F0078
:1022600014427800814F5200F6FF3200CFAA970047
:10227000D508900060C6B3002FDB9700804F530055
:102280000300320060C4B300804F530004003A00E2
:102290007FA09700008040008006E8000A00370019
:1022A0008001EB0050C6B300AFDB970080CF530036
:1022B0000300320050C4B30080CF530001003A0045
:1022C00013002000838640008D0F570001003D0061
:1022D0008E0678000D00E000240035008E8F560039
:1022E00006003D006FA89700E0C07E0092C3B300D7
:1022F00040C3B30080CF500001003C0002C3B300D4
:102300008D00E900EFA9970063C07800824F50006C
:1023100006003A008D06E9008100E9006FAA9700E7
:1023200064C07800824F5000FAFF320090C3B300BF
:10233000804F510004003A00EFAA970065C0780072
:102340000040E80080F278000100E00007003D0056
:102350006FAB97000603E900E6AF9F008D06E8002B
:102360007FA097000000E800F0A79F007FA29700E1
:102370008D0178006FA99700AFD897004FA89700FC
:102380000E0107004F0778004F06BE004F05BE0044
:102390004F04BE00EF04B100000006000000E000A2
:1023A00003003400D2020700E10F400001003A00B0
:1023B0000000EB00000006000000E00036003200E4
:1023C0000081E90012027800E30F5200320036006B
:1023D0000408A30030003A00616980000100E000B9
:1023E00002003200810F5100030031000108780023
:1023F000626988001D00370081017800110090009B
:102400000000E00008003200820F5000060031009A
:1024100080017800100090000000E000020032000F
:10242000820F5000FAFF39009300780001804100CC
:10243000800F510018003900820F500003003A004D
:102440008489400003017800080037009300900061
:102450000100E0000300320004004100808F5000C2
:102460000D0039001101980092019800920090002F
:102470000100E000080032009201780003004100F2
:10248000810F500004003A002A2DEF00108941000E
:102490001000900010019800000006000001780074
:1024A000000020000000E000080032000000800072
:1024B0000000E000050032000000E9000000880094
:1024C0000000D0000100800002B07800000006008B
:1024D000889FBE00800478000104780031009000DD
:1024E0000000D0004501DE00F07F2000800F510089
:1024F00010003A00800CEB00310090006F0060008B
:1025000008003A00210090000000E00005003A00B9
:10251000110090000000E00002003A001100E0000D
:1025200002003200200020001500370010002000BB
:10253000130037000200E00005003C0001007800B5
:10254000CF010700000178000000E0000A003C0015
:1025500038009000F10028000100600001FE230017
:10256000010070003004980020C02F00800C410052
:102570000080EB0002003700800CEB000000EB0055
:102580004F04BE0000000600881F78008A9FBE002E
:10259000000478000205BE00300190000200D00067
:1025A000C500DE00F07F2000808F50000C003A0054
:1025B0006F00610008003A00280090000000E00071
:1025C00005003A00180090000000E00002003A0008
:1025D0001800E0001C003200200020005D003700E1
:1025E0000100E00006003A0008007800A40107009E
:1025F000800078000000EB000100E00055003C0086
:102600006108B9000A0540008B854800E07F200082
:10261000800F5500E08F5D000D0034003800900001
:102620006022B8000600200007FF2F000000E00035
:10263000030035006022B8000600200007FF2700D5
:10264000049CBE000694BE0010002000410037002C
:10265000B8009000E00F5500E08F5D0005003400E9
:10266000F000280000806000C450DD000100700010
:102670003600370000002800808260006F80600014
:102680000040A0003004980061055500E0855D0021
:10269000C0FC2F00F1FF2F00800F5500818F5D00DF
:1026A00006003D00350498000000EB00200498006F
:1026B00010049800000CEB00260037000A02780096
:1026C000F00F45000B003C0018009000000C780053
:1026D0002800900010049800380090002004980012
:1026E0000000EB003004980070024200F00F42003E
:1026F000F5FF34000402EA001200320018017800ED
:102700000411DE00F0011200180090008300DD00CB
:10271000010C71000400DE00280190008310DD0030
:1027200001007000100498000411DE0038009000D1
:102730008301DD0003017100220498000400DE0023
:1027400030049800380090000500700030049800B4
:102750000080EB004F05BE004F047800000006002B
:102760000400FA00889FBE008A9FBE008C9FBE00B6
:1027700080BF9F0091BF9F000206BE0001020700BC
:102780000001BE000004BE000C00BE00A40407004F
:102790000FB997009FB99700000551008185590036
:1027A0000800BE000A01BE004F06BE004F05BE0075
:1027B0004F04BE000080FA00000006000A00FA0084
:1027C000889FBE008A9FBE008C9FBE0000047800D8
:1027D00001457800820578008304780004067800BB
:1027E0000300E00002003C00190020006BD820002C
:1027F00060C6B300804F55000E00320060C4B300C5
:10280000804F55000B00320070C6B300804F55005A
:102810000300320070C4B300804F550083003A00BB
:10282000E40F46008100350058089000800F5600E4
:102830007E003D000C06E80060C6B300804F5500E6
:102840001000320060C4B300804F55000D0032000C
:10285000081090000038A30004003A0058089000C7
:10286000808F540001003D00590C980058089000DA
:102870000C005000500C980002003B000000EB00E0
:10288000500C98000C00E00027003C00F2014400CE
:10289000130178006800900001C3B3000170790053
:1028A0000201E80082097800580890000000E0006A
:1028B00003003C00081090000038A3000400320020
:1028C000E8009000E0C2B300807079008209E8005F
:1028D0000C00EA00D8089000808F500001003D00F5
:1028E0000106EA000C00EA00200C98000C80400071
:1028F000500C9800890F500001003D0080047800C2
:10290000680090009808900001004000390C980081
:10291000090178008B00780008F70700580890003C
:10292000090050001A003700E800900018089000D5
:102930008C8F540018003D00008040000901780091
:102940008B007800FDF60700180890000901400090
:10295000120C980009005600200C980058089000AE
:102960000000E00003003C00081090000038A300C5
:1029700006003200E8009000E0C2B30080707900E9
:10298000380890000000E800300C980058089000CB
:10299000400C9800A3003700008040000C01780034
:1029A0008B007800E5F60700180890000C00400046
:1029B000100C98008C845400580890000000E0002F
:1029C00003003C00081090000038A300060032000D
:1029D000F20144009300780068019000E0C2B30067
:1029E00000F178008109E80058089000890F500034
:1029F00001003D0080047800680090009808900075
:102A0000010040008C80450009017800CBF60700EA
:102A10001808900009004000100C98005808900019
:102A200009005000200C98007E00370070C6B300EB
:102A3000804F55000300320070C4B300804F550032
:102A400014003A0058089000808F540004003D00A4
:102A5000081090000038A30001003A00590C9800BB
:102A6000580890000000E900500C980002003B005C
:102A70000000EB00500C980051C6B30070C6B300C4
:102A8000804F55000100320051C4B3000145780069
:102A90000900370010C6B300804F550002003A000D
:102AA0000AC7B3000400370010C4B300804F5500BC
:102AB00001003A000AC5B300F20144001301780096
:102AC000680090003B7079000201E80082097800FC
:102AD000580890000000E00003003C00081090003F
:102AE0000038A30004003200E8009000E0C2B30008
:102AF000807079008209E800580890000000E0002A
:102B0000100034008904E900890F500001003D00E5
:102B10008004780068009000980890000100400050
:102B2000090178008B00780084F6070018089000EF
:102B300009004000100C980058089000090050004F
:102B4000200C9800E8009000180890008085400054
:102B50008A5D78008B06E8000C00E0000400350078
:102B6000B0C2B300804D78008D05780004003700B6
:102B7000D0C2B300804D78008D0578000C06EA00C5
:102B80008004EB000C00E00009003400A1002000EC
:102B90000C0078008D0007007681540001F17F0061
:102BA000000678008904E8000000E000F7FF3C0020
:102BB000E18F540009003C0050C6B300804F55001F
:102BC0000300320050C4B300804F550003003A00A8
:102BD00000C3B300805E78008D0578000900E00036
:102BE00002003A0000C3B300805D78000900E000F5
:102BF000070034008904E900F680540061C07F00BA
:102C000002C3B300825D40000900E000F9FF3C0010
:102C10006800900098089000010040000080550076
:102C2000300C98000810900074006000F00F500005
:102C30000E003A00780090009808900001004000D3
:102C4000A808900001004000B80890000100400072
:102C5000C80890008100400078089000808F5000E4
:102C600002003D0001005000000C98004F06BE001D
:102C70004F05BE004F04BE000080FA0000000600B1
:102C8000000278003000900001002800010360007D
:102C9000150020006F0060003002980008003A0024
:102CA000240090000000E00005003A0014009000AD
:102CB0000000E00002003A001400E0003E00320094
:102CC000340090000000E0000B003A002400900067
:102CD0003002980014009000200298001400780040
:102CE00010029800000AEB00F082520034009000BD
:102CF0000000E000F5FF320034009000EF0F5000BC
:102D000014003E008001D000A40090004F08DE00B7
:102D100080817100330298008100D000140190007E
:102D20004F10DE0080807000210298000201D00068
:102D3000940078004F08DE00000171001202980034
:102D4000010AD0008502E90003007800EF8F5100EE
:102D5000ECFF3600B4019000FF8F510013003600E5
:102D60001401D10014009000CF00DD00010A7100B1
:102D70000000D100A40090004F09DD0002007000A7
:102D8000100298008100D1004F18DD008080700093
:102D9000210298000300D100300298008502E8006B
:102DA00080017800FF0F5000EDFF3E0034009000DE
:102DB0006F00600030029800340090000600700040
:102DC000300298000500780000000600010178003C
:102DD00000027800110009000200D8000002FD0086
:102DE0000491B900820250000400BE0000000600F9
:102DF0000A00FA0000027800C3202000E52020002D
:102E00000721200046212000E20F50001B003E0059
:102E1000406A8000E10F500004003200632120006E
:102E200085212000A7212000E621200013409000EA
:102E30000078A30002003A00000BEB0013F0A000A2
:102E4000154090000028A30001003A0015A0A00042
:102E5000820178000200E00010003200154090006E
:102E60000008A300FDFF32003100FB00800B78005A
:102E70008301E900F9FF3A00080037003000200024
:102E8000B0BF9F00C4BF9F00D1BF9F00E2BF9F00A3
:102E90006A80570000C0DA006FB99700020078001E
:102EA0000080FA00000006000A00FA00110020006D
:102EB000B1BF9F00C0BF9F006A80570000C0DA000A
:102EC0004FB897000080FA00000006000A00FA00E0
:102ED00051002000B1BF9F00C0BF9F006A80570013
:102EE00000C0DA005FB897000080FA00000006001A
:102EF000889FBE00800478004A0DE20005003A0079
:102F00000000EB00100007008080EB000000E000F4
:102F10000A003500586A8000880078000900E00047
:102F20000600320009004400070007008080EB0023
:102F30000000E00001003500880078000100780002
:102F40004F04BE0000000600800078000001EB0086
:102F50000000E00003003A0080D82000506A88009A
:102F60000600370000172100808F500002003E004D
:102F7000516A8800010037000081EB0002007800F0
:102F800000000600839F68000100E00002003D0091
:102F900060001000E08018000300E00002003D0027
:102FA00060011100E08119004B0007004F00E000B4
:102FB00002003B0060001000E080180000000600E6
:102FC000889FBE008A9FBE008C9FBE000404B8008C
:102FD0000506B8008904460060854E000606B80064
:102FE0000A054600E0854E000706B8008B0546003E
:102FF000040EB800890446000A854E00050EB8008C
:103000000A0546008B854E00060EB8008B0546006B
:103010000416B8000A0546008B854E000516B80058
:103020008B054600041EB8008B0546000800BE0054
:103030000A01BE004F06BE004F05BE004F04BE0091
:10304000000006000800FA00889FBE008A9FBE00AC
:10305000170007000605BE000404BE00E00F520082
:10306000E08F5A00E00F5B00E08F5B0008003D003E
:103070000400BE000601BE002A0007000205BE00D3
:103080000004BE000F00070026000700080007002C
:103090000802BE000A03BE000A000700C8FF0700BE
:1030A0004F05BE004F04BE000080FA00000006007D
:1030B000E0B79F00F1B79F0082BF9F0093BF9F00C2
:1030C000000006006FB09700FFB097000FB997009F
:1030D0009FB99700000006006022B8000602200099
:1030E0000000D0008180D2000482D2008582D2000C
:1030F0000000A0000202520083825A0003003B003D
:103100000202420083824A000000A1000603E90097
:10311000F3FF3A0000000600EFFF07000400BE00C6
:103120000000060060001000E08018006001190037
:10313000E081190000000600810378003E020700CC
:103140000001BE006000B8000478A30013003A003C
:103150006220E10015003E000D0039008301D1001E
:103160000281D3008180D3008301D1000281D3008A
:103170008180D3008301D1000281D3008180D300FC
:103180000538B000C42ADD00F300B200838172006C
:1031900007F0A70003F0A00000000600F3FF2700DF
:1031A000F2FF2F006110B900FBFF370003FF27007B
:1031B000F7FF3700881F7800000478005001BE0038
:1031C0004000BE000000420081804A0002014B0026
:1031D00083814B00009CBE000294BE00DC0007000F
:1031E00003003100480090000000E800400498000F
:1031F0004F04780000000600889FBE00000478009D
:103200008004EB005001BE004000BE00D00007006B
:103210000100310019002000040050008580580092
:103220000601590087815900009CBE000294BE002F
:103230004800900009005000400498004F04BE0070
:10324000000006001200FA00889FBE008A9FBE00A0
:103250008C1F78000205BE000004BE00F4B79F007A
:1032600085BF9F0096BF9F00A7BF9F000000EB0097
:10327000E0B79F00D0B79F00C0B79F00B0B79F00D6
:10328000A0B79F000006EB005FB197006FB09700FA
:103290008000D0000000E00015003D00E1B79F0075
:1032A000010078000200E00001003D000000A000E5
:1032B000AC00070001003D000000A000AF000700C7
:1032C00001003D000000A000B200070001003D0029
:1032D0000000A0008100070001003D000000A000E8
:1032E000B20007007C805700B2FF070014003700CF
:1032F000E1B79F00010078000200E00001003D00FE
:103300000000A0009700070001003D000000A000A1
:103310009A00070001003D000000A0009D0007008A
:1033200001003D000000A0006C00070001003D000E
:103330000000A0009D0007007C805700AEFF070042
:103340006FB097000000E00007003500100020007B
:10335000010020006011B80008047000898470002A
:103360000A0571008B8571000C06E800F00320004F
:10337000800F5600C4FF34006FB097000000E000DB
:1033800006003D007FB297008FBA97001FBB9700E1
:10339000AFBB97007C80570086FF07000802BE0085
:1033A0000A03BE006FA897000000E00004003A0086
:1033B0002FB29700BFB297004FB39700DFB39700CB
:1033C0000400BE000601BE004F0678004F05BE0097
:1033D0004F04BE000080FA0000000600881F78003D
:1033E00018002000881F780096FF07008F87E900EB
:1033F0004F04780000000600801FEB0091FF0700DB
:103400008F87E900000006000800FA00889FBE00D0
:103410008A9FBE008C1F78006E00070005003D00EB
:1034200043000700300007000C003D003300070098
:103430000B003700E00F5200E08F5A00E00F5B00F6
:10344000E08F5B0006003D000400BE000601BE00E8
:1034500034FF07000205BE000004BE001C0020006F
:103460002C000700DDFF07000C00E0000100320027
:103470002CFF07004F0678004F05BE004F04BE002A
:103480000080FA00000006000800FA00889FBE00D5
:103490008A9FBE008C1F78004E00070002003D008E
:1034A0001C002000220007000F00070001003D0063
:1034B0001200070017000700CFFF07000C00E00014
:1034C0000100320017FF07004F0678004F05BE00CD
:1034D0004F04BE000080FA000000060090B79F0075
:1034E0000100D00080B79F00E00F5400E08F5C0027
:1034F000E00F5D00E08F5D00000006000800BE00E8
:103500000A01BE0007FF07000205BE000004BE005E
:10351000000006000802BE000A03BE005FB097006C
:10352000EFB097007FB197008FB9970000000600B9
:10353000FCFE07000100070000000600B0B79F0076
:10354000C1B79F00D2B79F00E3B79F0000000600FD
:103550000400E1000588E1000690E1000798E10021
:1035600000000600C0B79F000200D000B0B79F0067
:10357000AFB097000100E00000000600B0B79F0068
:103580000100D000A0B79F009FB097000100E000AD
:1035900000000600A0B79F000100D00090B79F0078
:1035A0008FB097000100E0000000060080B79F0088
:1035B0000804D0008984D2000A85D2008B85D2000D
:1035C0005FB29700EFB297007FB397008FBB970071
:1035D00000000600D9FF07000605BE000404BE0077
:1035E0000006EB00E00F5000E08F5800E00F59009C
:1035F000E08F5900000006008F1FD1002301070053
:103600008F87E9000000E000000006001400FA00C7
:10361000889FBE008A9FBE008C9FBE000004BE0033
:103620000205BE00680047000A90BE000890BE0078
:103630003F0107000070A7000BF0A10030432000FD
:103640009E02900080825200B0FE2F000028E10010
:1036500011003D00B0FC2F000028E10015003400EF
:103660001E0990008E0890007E0090000501B000B9
:103670000201D1008180D3000080D3008502E800E0
:10368000FBFF3A000B00E00064013B00600010000B
:10369000E080180061013700F0FF2F00F1FF2700E4
:1036A0000B00E0005D013B0001002800000020004D
:1036B0005A0137006000B800580137004F89DE001A
:1036C000820178005A01370007F0A2008F0137000D
:1036D000809FEB00ED0007008F87E9000000E0000D
:1036E000000006002800FA00889FBE008A9FBE00E6
:1036F0008C9FBE0003866B00340107000028A300E6
:1037000064003A000128A30067003A000008A30003
:1037100062003A000108A30065003A001E00900014
:10372000BE08900081064000ED3FB100F4805700D4
:10373000EE019000111AB8008E099000311BB800FC
:103740009E099000311CB800511DB800F485570047
:1037500046000700FE0190003A0007008B85E80054
:103760003E0007008E09900040000700EE01900027
:10377000340007008B85E800380007008E099000B0
:10378000400007009E0990001B18B8008904400003
:103790000A854800FE019000340007008B85E80090
:1037A00038000700EE019000300007008E099000FD
:1037B0001B18B800890440000A8548000A98A30035
:1037C00008003A000402420085824A0006034B00CA
:1037D00087834B0008044C0089844C000A054D0087
:1037E0008D06E90084827200850273004C3ADD0088
:1037F000850272000100320015002000443ADE000C
:103800001400B2004538DE00CB45DD000B0070002F
:10381000C540DE00CB4DDD008B8070004549DE00E9
:10382000CB55DD000B017100C551DE000D037800A2
:10383000B301070003F0A1000CF0A70003F0A00003
:10384000F60037001B18B8008502400006834800C8
:10385000E0834B0060044C00070037001B18B800E1
:103860000603400087834800FAFF37001B18B800A2
:103870008703400008844800E0844C0060054D0048
:10388000000006001B18B8000804400089844800A6
:10389000FAFF37000108A300DD003A005800BE001F
:1038A0005801BE00E3FF37000008A300D8003A002B
:1038B00009047800F9FF37002800FA00889FBE004D
:1038C0008A9FBE008C9FBE0003866B00BF0007006E
:1038D0006400E100440032006408E1004A00320064
:1038E0006100E100460032006108E1004900320059
:1038F000EC0647006000B8003D02BE003D03BE007C
:10390000F48657006011B8003D04BE003D05BE00BE
:103910007D0320000B0037000000A0008D06E900A9
:10392000130032000402420085824A0006034B0065
:1039300087834B000000400081804800020149005D
:10394000838149000802520089825A000A035B0001
:103950008B835B00F0FF3B000802420089824A0033
:103960000A034B008B834B008D06E900EDFF3A0004
:103970008482720086827200F707B200878272002A
:1039800001003200150020001E0490003E0B900044
:1039900006035400E63FB0000368A30007003200AE
:1039A0000000A7000500A0008301D1000281D30020
:1039B0008180D3000080D3000603E8008301D1009A
:1039C0000281D3008180D3000080D3000002EB008D
:1039D0000482D2004A01070003F0A1000CF0A70006
:1039E00003F0A0008D003700640247006408E10086
:1039F000870032003400BE003401BE00F6FF3700FD
:103A00006108E100820032006011B8006000B80077
:103A1000F1FF370003FF270002002000FBFF370003
:103A2000020AB900001BB9000200B8008100420080
:103A30008100430000000600C70ADE00F107B20063
:103A4000F50FB20008003200E1CF42000200320060
:103A50000170A00024000500810F700001003200F9
:103A60000408050044000500810F700002003A00C0
:103A7000140005008502E9000000400081C04800F4
:103A8000FCFF3B000170A00024000500889FBE00E1
:103A90008A9FBE008C9FBE000404BE000605BE00C7
:103AA000809FBE00829FBE0041010700040678008F
:103AB0000800BE000A01BE003D0107008406780030
:103AC0004F03BE004F02BE008D4F76007FB09700BF
:103AD00013003300F0FF2F008B8F6B0006003B00BC
:103AE0000D0666000C00A7000A00370007F0A600CC
:103AF000100020000A003700880F5200898F5A00FA
:103B00008A0F5B008B8F5B000300390010002000E0
:103B100001003E000000200007F0A7000000EA00BE
:103B20004F06BE004F05BE004F04BE000000060059
:103B3000800078005002BE005003BE004439DE0011
:103B4000F700B200F37F200003016100090032009A
:103B50000218E10016003A0085017200830173002B
:103B6000838173000008200015003A004000200007
:103B70001300370085017200830173008381730095
:103B800005003A0004A8BE0006A8BE0010002000F0
:103B90000B0037000201E9000402420085824A005E
:103BA00006034B0087834B000748A300F9FF320050
:103BB0000740A00004A8BE0006A8BE002000200008
:103BC00080009800920098000000060068044700FA
:103BD0000294BE000094BE00FC0447008694BE0020
:103BE0008494BE0009007800D1FF07000800780027
:103BF000CFFF070099007800814F70000B003B0059
:103C00000800BE00FC0007004F00B10003003700B1
:103C1000F3FF2700F2FF2F006110B9004F06BE002E
:103C20004F05BE004F04BE000080FA0000000600F1
:103C3000889FBE00830478000300E0002C0035005C
:103C400003003C0000827000040271002600320074
:103C500036432000C50020008383CF000A003900CE
:103C60000541B1008283CF00070039000541B10052
:103C70008183CF00040039000541B1008083CF006B
:103C8000010039000541B10085C353006022B8002E
:103C9000120032000A003B00848272006102600060
:103CA0008301D1000281D3008180D3000080D30042
:103CB0000603E8008743E800F7FF3A0007003700F3
:103CC00000004000818048000201490083814900D2
:103CD0000603E9008743E900F9FF3A00880007007E
:103CE00009F0A70003F0A0004F04BE00000006008A
:103CF00060001000E080180060011900E0811900E8
:103D0000D3FF3B00033E2C00F7FF37002800FA00EA
:103D1000889FBE008A9FBE008C9FBE000706780069
:103D2000878669000C003B00030478008704780054
:103D300008F0A10009F0A100840F5000858F580001
:103D4000860F5900890F5C00030033000CF0A200BD
:103D500001003A000CF0A1009CFF07006400E100A4
:103D60005F003200780147006408E1006100320022
:103D70006C014700748557003200BE001201BE007E
:103D80003A04BE001A05BE001E039000BE0A900051
:103D90008503530006003D000004FD008104FD0082
:103DA0000205FD008305FD008703EA000503780096
:103DB0000DF8A3000400320060041400E0841C002D
:103DC00060051D00E0851D006022B8007D03200015
:103DD0000D38E1008006EB000B0039004433DD00B4
:103DE000F300B2008301730039003700848272004F
:103DF0000D027800E10664008B85D1000A85D300AE
:103E00008984D3000884D3008703E900F7FF3B00CF
:103E100008004000898048000A0149008B81490060
:103E200004003B0060001000E080180060011900F1
:103E3000E08119000358A300090032008D8272004E
:103E400084827200610260008301D1000281D3008C
:103E50008180D3000080D3000603E8001B003700F8
:103E60000348A30017003A000600E00017003400E2
:103E70000603E9000D00A30000004800818048000F
:103E800002014900838149000348A3000F003A0062
:103E90000600E000090034000603E90000004000CD
:103EA00081804800020149008381490001003A00F5
:103EB0000003EB000348A300F5FF32006022B800C6
:103EC0000200370084827200618266000C000700E5
:103ED00003F0A1000CF0A70003F0A0004FFF370093
:103EE000640147006408E10002003A000DF8A300F5
:103EF00047FF3A003200BE001201BE0047FF370004
:103F00001800200057002000080453000D003D0059
:103F10000600200097FC2F000740E1001E0034003F
:103F200084827200610260008301D1000281D300AB
:103F30008180D3000080D3000804E800F8FF3A0035
:103F4000470020006104600005047400040464005C
:103F50000D00320061004000E0804800600149002F
:103F6000E081490003B8A500070032000603E8001D
:103F70006538E10004003A008301D1000281D300DA
:103F80008180D3000080D300F87F20000830E1005A
:103F900003003500080378006000B8006011B80025
:103FA0004433DD00F300B20083017300000006001B
:103FB00005FF270005826100070032000428E100A8
:103FC00001003200240005000600070001003A004D
:103FD000440005000408050002000700F9FF3A004C
:103FE000140005006F82610081027000850271007B
:103FF0008502720000000600E48240001078A300F1
:1040000007003200640240001178A3003400BE00B3
:104010001401BE00040032000330A70000000600B7
:104020003500BE001501BE000330A00000000600F0
:104030000200FA00881F78004079280051A820006B
:10404000304588004145880030F92E00414121006B
:10405000504588006145880020002000000F78004E
:10406000D00120009E0F100018003C009E00780038
:10407000400020000008B800628A200002044000CE
:104080001E0078006103B90003AF2D0063009000AB
:104090000032B8007300900000B0B900050178004C
:1040A00000014100630090000780B9000001410059
:1040B000820278004079280051A82000001C4200AC
:1040C00001944A001E0FE800E5FF370010002000B1
:1040D000204988000000EB003049880020002000C3
:1040E000404988000000EB00000F7800D00120005C
:1040F0009E0F100008003C001E0078000000D00059
:10410000A2922000820040000000EB0080087800AE
:104110001E0FE800F5FF37000000EB00304B880071
:104120000000EB00404B88000000EB00604B880073
:104130000000EB00504B880020002000704B8800EE
:10414000004B2000804B8800800C2000904B8800A2
:10415000B0042000A04B880020022000B04B880053
:10416000D0012000C04B8800C0012000D04B880047
:10417000E027280001002000F0488800014988005D
:10418000D04E21001049880020002000E04B88001C
:1041900010002000F04B880010002000004C880028
:1041A0000000EB00104C880030002000204C8800FC
:1041B00000502900A1AB2000404C8800514C8800E1
:1041C000509D210001002000604C8800714C880047
:1041D0004008200001002000804C8800914C88009D
:1041E0000078200001002000A04C8800B14C88001D
:1041F0007001200001002000C04C8800D14C8800D4
:104200007001200001002000E04C8800F14C880083
:1042100020032000004D880030C0B300A2E9B700A1
:1042200030C0B300A3E9B70010C0B300A4E9B700E1
:1042300010C0B300A5E9B70010C0B300A6E9B700ED
:1042400010C0B300A7E9B70010C0B300A8E9B700D9
:1042500010C0B300A9E9B70010C0B300AAE9B700C5
:1042600010C0B300ABE9B70010C0B300ACE9B700B1
:1042700010C0B300ADE9B70013002000428A20004F
:10428000E11F2F00F0072000FB0F070020458000F2
:104290000000E8002045880012002000E11F2F00E8
:1042A000F00720000110070013002000E21F2F007C
:1042B000F1072000408A20001D1007004F047800FD
:1042C0000080FA00000006000400FA000000EB0085
:1042D000304C88000000EB00000F78000007200041
:1042E0009E0F100024003E00F00620009E0F1000DC
:1042F00008003E001E0078000000D000628A200006
:1043000082004000304C800011004000304C88009A
:1043100003003700304C80000000EA00304C880079
:104320001E0078000000D00002002F008200400034
:1043300012002000F0072000DC0F07001007980093
:104340001E0078000000D00001002F000101400095
:104350001E0078000000D000618A200001004000AB
:1043600013002000F1072000F10F0700100798004C
:104370001E0FE800D9FF37008609F8001E019000E3
:10438000821F78001E007800801F780040BB2D003F
:10439000801F780009F00700E88757000080FA00C6
:1043A000000006000600FA000000EB00200798005D
:1043B0000000EB00000F7800000720009E0F1000A7
:1043C00015003E001E0078000000D000618A200029
:1043D000010140001E0078000000D00003002F0003
:1043E0008300400013002000F0072000A20F070008
:1043F000100798001E0078000000D000628A20009C
:10440000820040002E00900011004000200798001C
:104410001E0FE800E8FF370013002000428A20004A
:10442000E11F2F00F0072000930F07002E009000DF
:104430000080FA00000006000400FA000000EB0013
:10444000904D88000000EB00000F78005001200024
:104450009E0F100024003E00410120009E8F10009E
:1044600008003E001E0078000000D0008298200066
:1044700082004000904D800011004000904D880067
:1044800003003700904D80000000EA00904D880046
:104490001E0078000000D00002102F0082004000B3
:1044A00012002000F0072000800F0700100798007E
:1044B0001E0078000000D00001102F000101400014
:1044C0001E0078000000D00081982000010040000C
:1044D00013002000F1072000950F07001007980037
:1044E0001E0FE800D9FF3700B209F8001E01900046
:1044F000821F78001E007800801F7800D0BD2D003C
:10450000801F7800ADEF0700E88757000080FA00B1
:10451000000006000600FA000000EB0020079800EB
:104520000000EB00000F7800500120009E0F1000EB
:1045300015003E001E0078000000D0008198200089
:10454000010140001E0078000000D00003102F0081
:104550008300400013002000F0072000460F0700F2
:10456000100798001E0078000000D00082982000FC
:10457000820040002E0090001100400020079800AB
:104580001E0FE800E8FF37002E0090000080FA00C0
:10459000000006000E00FA00000F780011079800D6
:1045A0009E00900040062000008AB9001E0078009E
:1045B0006101B9000400BE0072FA070030079800DC
:1045C0004107980042062000030020003E009000B2
:1045D000CE009000000051008180590050079800E3
:1045E000610798005E009000EE009000E00F500020
:1045F000E08F580004003C00100020000100200063
:104600005007980061079800100320009E0F1000CB
:10461000150034003E009000CE00900042062000BD
:104620000202B8000001EB000283B9000501780026
:1046300006014100430620000388B9000001410043
:104640008202780000712200010020000400400076
:10465000858048005E019000EE01900049FA070055
:1046600020079800020037000000EB0020079800A8
:104670002E0090000080FA00000006000400FA00FE
:10468000B0002000CD0D0700CF80DE00A24C8000DE
:104690000202B800B24C80000283B9000501780024
:1046A00006014100A34C80000198B90000014100BF
:1046B00082027800048FBE001E00BE004008DE00AB
:1046C00001002000B0438800B0438000110A0700B9
:1046D0000080FA00000006000200FA00C1438000DA
:1046E000207520000088B9004008DE00010020008D
:1046F000F0448800F0448000060A07000080FA00B9
:10470000000006000000FA003408E20002003A004F
:10471000F1FF070001003700D8FF07000080FA0012
:10472000000006000200FA003408E20026003A0009
:1047300070C02D00040B070031448000E04C800065
:10474000000AB80031448000F04C80000088B900B5
:104750000501780000014100E14C800040448000E8
:104760000088B900000141008202780040A8DE0004
:10477000CF80DE00000F7800504480009E0F1000B4
:10478000040034001E0078005044880060042000BB
:1047900060448800604480000000E90060448800B4
:1047A0008C08E20004003A006004200060448800A5
:1047B0001E0078005044880071072000504480009B
:1047C0001A0C070006003700B0C02D00DE0A0700F3
:1047D0000000EB0050448800600420006044880022
:1047E0000080FA00000006000000FA003408E20031
:1047F00018003A0090002000700D0700CF80DE0006
:10480000624C80000202B800724C80000283B90042
:104810000501780006014100634C80000198B90051
:10482000000141008202780040A8DE00CF80DE0057
:10483000E043880040C12D00C30A0700210020008A
:10484000E0438000F90B070070C12D00BE0A07008D
:104850000200370090C12D00BB0A07000080FA005B
:10486000000006000200FA000000EB00000F7800D4
:10487000A00020009E0F10000C003C0042B22D0052
:104880009E007800400020000008B80000014100B0
:10489000D0408000E1408000B20F5000A28F58004D
:1048A000020035001E0FE800F1FF37001E007800FF
:1048B000604188000080FA00000006000000FA0055
:1048C000E8FF070060418000219A200001004000BD
:1048D0001080FB004E00DD005041880001B52D0026
:1048E000604180000000D00001004000100078000E
:1048F000A04D8800A14D80005041800000807000D4
:10490000A04D8800D2408000E3408000B0602B00C2
:1049100001B62000800F5100818F5900040034003F
:10492000A04D80000108200001007000A04D88000B
:104930008009E20004003200A04D80000104200044
:1049400001007000A04D88006A09E20004003200F6
:10495000A04D80000102200001007000A04D8800E1
:104960006C09E20006003200004C8000E10F5000AC
:1049700003003A00A04D80000040A000A04D880038
:104980006809E20003003200A04D80000030A00062
:10499000A04D88006E09E20003003A00A04D80009F
:1049A0000020A000A04D8800104180000000D00031
:1049B000A19220000100400011002000908F100003
:1049C00003003200A04D80000010A000A04D880020
:1049D000104180000000D000A192200001004000A2
:1049E00011002000908F100003003C00A04D8000BB
:1049F0000000A000A04D8800A04D800021110700FC
:104A00000080FA00000006000200FA00000000002A
:104A1000CFC2BF000080FB004600DE000080FB002C
:104A200061006000E10F50005C003A00D0002000FF
:104A3000E20C0700C0438800C0002000DF0C070024
:104A4000D0438800C1438000C04380000088B90083
:104A5000F043880001448800D1438000D0438000A7
:104A60000088B9001044880021448800F243800087
:104A70000344800010448000214480000000510065
:104A80008180590030448800414488000040EB0098
:104A90006D0807001BFF070070C02D002A0A0700E1
:104AA00031448000E04C8000000AB80031448000AE
:104AB000F04C80000088B900050178000001410039
:104AC000E14C8000404480000088B90000014100B2
:104AD0008202780040A8DE00CF80DE00000F780060
:104AE000710720001E007800500B070000C4B300BF
:104AF0005508070020C22D00130A070060418000FE
:104B0000219A2000010040001004E00003003A0058
:104B100000022000E509070002003700D002200053
:104B2000E209070060418000219A20000100400056
:104B300010407800920B0700E0C22D00020A070027
:104B400060418000219A2000010040001080FB009D
:104B5000000F7800A0002000700D07001E0F10004D
:104B6000300020009E0F10000200340030002000B2
:104B7000000F78001E00E00002003D000000EB0086
:104B8000000F780060418000219A20000100400061
:104B90001E48780049FF07009DFF370026FE0700EA
:104BA000540D07000080FA00000006000000FA0023
:104BB0003208E2000200320093FF0700470037008E
:104BC000604380000000A200604388006C08E2009F
:104BD00004003A00014D8000C0F62100830F070059
:104BE00003003700014D8000108F21007F0F070068
:104BF0001F080700004B200060678800CFC2BF007D
:104C00000080FB004600DE000080FB0061006000C9
:104C1000E10F500025003A000040EB000A080700B1
:104C200060678000C2122000110009000280D800D5
:104C3000801F780020C32D00801F7800C0832000D3
:104C4000BFED0700E4875700C0832000BE090700BE
:104C500000C4B300FC0707006C08E2000300320048
:104C600050C42D00B80907000200370060C52D00B0
:104C7000B5090700EC0CE200E0FF3A00004D8000AF
:104C80008000D000E0552200580F0700CFC2BF00BF
:104C90000080FB004600DE000080FB006100600039
:104CA000E10F5000F9FF3200D4FF3700EC0CE200B6
:104CB0000A003A0084FD0700AC0E070070C62D0004
:104CC000801F7800BDED07008F87E90020002000DD
:104CD000680C0700CFA2A900FFFF37000080FA0090
:104CE000000006000200FA00E107070040C92D009D
:104CF0009509070000C4B300D307070050CA2D0070
:104D000091090700750B07000000E0001100320058
:104D1000820B0700004F7800A1002000904F210077
:104D2000320F07001E4078005D0B070000C4B3007F
:104D3000C507070060CB2D00830907001E80FB001C
:104D40005A09070000CC2D007F0907001E4078009B
:104D50005C090700CFC2BF000080FB004600DE00F8
:104D60000080FB0061006000E10F5000E5FF3A00A9
:104D70000080FA00000006002600FA00889FBE00AE
:104D80008A1F7800F0F32F00001688000000EB0067
:104D90001016880030E72F00301688000000EB0066
:104DA00040168800E0012400601688000000EB0037
:104DB000701688000000EB00901688000000EB00E1
:104DC000A016880080E12F00F01688000000EB009C
:104DD0000017880000082100201788000000EB0061
:104DE00030178800CFA2A80040442500A004880006
:104DF000330E0700160D07006000B800FC0C07001A
:104E00004079280051A82000F90C070050552500D2
:104E100051552500204088003140880020032000A3
:104E200040678800C0D42100404088000000EB00AB
:104E3000504188000000EB00A04D880003100700DF
:104E4000A04D80000F10070091070700DA07070048
:104E50008707070050CC2D003B09070060AC2D00F0
:104E60003909070000C4B3007707070000CD2D0003
:104E700035090700ED0A0700DF18070010CE2D00E6
:104E8000801F78004DED07008F87E90060AC2D0092
:104E9000801F780049ED07008F87E90090CF2D0033
:104EA000801F780045ED07008F87E900D0AC2D000A
:104EB000801F780041ED07008F87E90020D02D008A
:104EC000801F78003DED07008F87E9000808F80093
:104ED000A0D22D00801F780038ED0700E48757002E
:104EE00020D42D00F0180700A50B070020D62D00B8
:104EF000150907000000EB005043880080BB20002C
:104F000060678800CFC2BF000080FB004600DE0063
:104F10000080FB0061006000E10F500020003A00BB
:104F2000EC0CE200F7FF3A00020E0700C11220006D
:104F3000E0552200AD0E070000C4B3004207070091
:104F4000B0D62D0000090700100020005043880053
:104F500020C72100711C27002040880031408800B4
:104F6000CFC2BF000080FB004600DE000080FB00D7
:104F700061006000E10F5000F9FF32000040EB00DB
:104F800031070700C0D72D00EF08070000C4B300A9
:104F90002D070700D0D82D00EB080700D9FF3700F8
:104FA0005CFD070030079800FEFC070040079800F2
:104FB000A408F8004E009000801F7800BE0090000A
:104FC000811F7800E0D92D00801F7800FBEC0700DE
:104FD000E88757003E0090000000E00003003A0020
:104FE0004E0090000000E000080032006F11070042
:104FF00050DE2D00801F7800F0EC07008F87E9005D
:105000000BFC07000CFD0700AFFC0700804B800085
:10501000F60D0700904B8000EE0D07002E0C0700E8
:105020000000EB00604388000000EB002043880094
:105030000000EB00304388000000EB0030438800A4
:105040000000EB00904188000000EB0080418800E8
:10505000324980001241880010418000E10F500069
:10506000020034000000EB00104188001141800074
:10507000400020000008B800638A200003004000C0
:105080001001BE00D2408800E3408800D04080007C
:10509000E1408000560C070042130700007D20000D
:1050A000740B0700F2060700A6160700A10D070003
:1050B000400120006F0B0700004D80008000D000F1
:1050C000904F2100490E07006A08E20001003200FB
:1050D0008F0F070000000000CEC2BF000080FB0061
:1050E0004200DE000080FB00610060000000E00084
:1050F00012003A000040EB00D306070060E12D00EB
:105100009108070000C4B300CF06070070E22D002D
:105110008D080700C3C2BF000080FB004400DE0012
:105120000080FB00610060000000E000EAFF3A0040
:10513000BFFB0700C0FC070063FC0700214C800098
:10514000800020000008B80083B62D0000804100D8
:10515000801F78008409F80080E32D00801F78000C
:1051600096EC0700E6875700204C80003D0A0700B8
:10517000204C8000E30F50000B003200214C8000D7
:10518000800020000008B80084B62D000000420016
:10519000801F78008409F80030E62D00801F780019
:1051A00086EC0700E6875700C3C2BF000080FB0003
:1051B0004500DE000080FB00610060000000E000B0
:1051C00001003A00C7FE07004D0A07004B18070010
:1051D000C8C2BF000080FB004600DE000080FB006C
:1051E000610060000000E0000300320010002000B9
:1051F000A0418800020037000000EB00A0418800B9
:10520000304980001041880040498000E20F500082
:1052100027003A00A0418000E10F500006003A004C
:1052200010418000E10F5000080034000000EB0046
:10523000104188000500370010418000E10F500048
:105240000200340010002000104188003049800026
:10525000E20F500009003A0060498000E20F500060
:1052600003003A0010002000804188001C00370035
:105270000000EB00804188001900370010418000D9
:105280000000D000A1922000010040002200200078
:10529000900F110003003A001000200080418800A8
:1052A0000F0037000000EB00804188000C00370041
:1052B000104180000000D000A392200003004000B5
:1052C00024002000900F120003003A00100020007C
:1052D00080418800020037000000EB008041880018
:1052E000104180000000D000A19220000100400089
:1052F00032002000900F11000F003A003408E20045
:1053000009003A00CA62A8003208E2000F003A0021
:105310001000200090418800014D8000904F210036
:10532000B20D070009003700CA62A9000000EB00B7
:1053300090418800050037003208E2000300320087
:105340000000EB0090418800CA62A9001A4DE200FB
:10535000650032006408E20063003A000040EB00A0
:105360001AEDB7006C08E2005E003A000A08E2009D
:105370001D003A0011418000400020000008B800E4
:10538000638A200083044000114180004000200017
:105390000008B800648A200004044000550B070090
:1053A0006103B90002AF2D002149800040002000B8
:1053B0000008B800800141001332B80013009000CB
:1053C00000B0B90005017800000141001300780029
:1053D0000780B9000001410082027800B81C420039
:1053E000A8944A001C0037001141800040002000B2
:1053F0000008B800628A2000820440001141800049
:10540000400020000008B800638A20000304400028
:10541000380B07006103B90082AD2D0061408000A8
:10542000400020000008B800800141001332B8009D
:105430001300900000B0B9000501780000014100A0
:10544000130078000780B900000141008202780053
:10545000B81C4200A8944A0011418000400020007E
:105460000008B800648A2000040140002040800049
:1054700031408000B20F1000A28F180008003400E5
:1054800011418000400020000008B800628A20001E
:105490000200400022408000334080000288BE00AD
:1054A00011418000400020000008B800638A2000FD
:1054B000030040001000BE00E00F5000E08F5800D5
:1054C00009003D0011418000400020000008B800A4
:1054D000648A2000040140006000B8000089BE001A
:1054E00001003700030B070011418000400020003D
:1054F0000008B800628A2000020040001001BE00CF
:10550000D2408800E3408800114180004000200024
:105510000008B800638A2000030040001001BE00AC
:10552000F2408800034188006609E200270032004B
:10553000F0002000210A070020079800AE0090002C
:1055400010832000808F5000050034002E00900052
:10555000E37C2F0003004000200798000B00370079
:10556000AE009000E07C2000808F500005003C00E1
:105570002E00900024832F00040040002007980094
:10558000020037000000EB0020079800AE009000FA
:10559000800120000088B900204188003141880046
:1055A000A0418000E10F500008003A002041800037
:1055B00031418000D2408000E34080000201400081
:1055C00083814800D2408800E34088001041800079
:1055D0000000D000A392200003004000240020001F
:1055E000900F120012003A003408E20010003A0056
:1055F000D2408000E3408000F048800001498000F4
:105600000000510081805900D0408800E1408800AE
:10561000F240800003418000F04880000149800092
:105620000000510081805900F0408800014188004D
:10563000D0408000E1408000ED0A07009FFC070099
:105640003408E2000D003A00104180000000D00054
:10565000A19220000100400012002000900F1100D4
:1056600003003C00D04B80004C0C070009003700C1
:1056700020032000490C070006003700704B800013
:105680000000D00043972000030040001000780085
:10569000420C07003408E20031003A00D00020003C
:1056A000C6090700C0438800C0002000C3090700E6
:1056B000D0438800C1438000C04380000088B90007
:1056C000F043880001448800D1438000D04380002B
:1056D0000088B9001044880021448800F24380000B
:1056E00003448000104480002144800000005100E9
:1056F000818059003044880041448800D1438000B3
:10570000C0438000A3FB0700C04488009C08E2005F
:1057100003003200E04480000000E900E04488001B
:10572000C1448000C0122000808F50000900340066
:105730009C08E20007003A000000EB0020438800CC
:10574000200020003043880010002000D044880052
:10575000050037000000EB00D0448800020037004D
:10576000800C2000E0448800E0002000930907003E
:1057700000458800010021000045800000805000A5
:10578000200798002E0090004015B00020079800D8
:10579000AE0090002E0090000088B900300F9800F5
:1057A000410F98003E089000CE0890004108DE00AE
:1057B00001002000200798002E0090007400400097
:1057C000200798002E02900044678800E04B80007C
:1057D000C04188008209E200120032003408E20071
:1057E00010003200B04380008080E8000045800057
:1057F0004680DE00808F5000060034006E08E20014
:1058000004003A00DD0B0700401F2000104588000F
:1058100009003700A208E20007003A00D30B070096
:10582000050037006E08E20002003A00D30B0700C3
:1058300001003700CD0B0700C3C2BF000080FB0092
:105840004500DE000080FB00610060000000E00019
:1058500051003A00803E2000606788006408E20042
:1058600007003A0030438000E40F500004003A0083
:10587000014D8000C0F621005C0C07000D003700D0
:1058800020438000E10F500007003A0040438000B1
:10589000EC0F500004003A00014D8000C0F62100DA
:1058A000520C070003003700014D8000108F2100CB
:1058B0004E0C070000000000C3C2BF000080FB00C8
:1058C0004500DE000080FB00610060000000E00099
:1058D00008003A00EC0CE200F7FF3A00014D8000AE
:1058E000A00020000088B90080007800C0F62100E8
:1058F0003E0C0700EC0CE20011003A00204380004F
:105900000000E8002043880020438000E10F5000A1
:10591000020034000000EB0020438800000000007B
:10592000C3C2BF000080FB004500DE000080FB001A
:10593000610060000000E000F9FF32001300370052
:105940006408E20009003A00304380000000E800EB
:105950003043880030438000E40F50000B003400D7
:105960000000EB003043880008003700404380000F
:105970000000E8004043880040438000EC0F5000E6
:10598000020034000000EB0040438800D909070002
:105990004006200037090700C3C2BF000080FB009B
:1059A0004400DE000080FB00610060000000E000B9
:1059B00031003A0020498000E20F500004003A0014
:1059C000014D8000C0F62100080C070003003700DD
:1059D000014D8000108F2100040C0700803E200044
:1059E00060678800C3C2BF000080FB004400DE0087
:1059F0000080FB00610060000000E00008003A0049
:105A0000EC0CE200F7FF3A00014D8000A0002000FE
:105A10000088B90080007800904F2100F30B070048
:105A2000EC0CE2000A003A00400020002049880007
:105A3000C3C2BF000080FB004400DE000080FB000A
:105A4000610060000000E000F9FF3200080037004C
:105A500020498000E20F500003003A0010002000AF
:105A600020498800020037002000200020498800DB
:105A700040062000FF080700CEC2BF000080FB00E8
:105A80004400DE000080FB00610060000000E000D8
:105A900016003A006609E20006003200014D80005F
:105AA000C0F62100D10B07000000EB00304B88004E
:105AB00005003700014D8000108F2100CB0B07003F
:105AC00010002000304B880040062000E908070045
:105AD000CEC2BF000080FB004400DE000080FB005F
:105AE000610060000000E000F9FF3200CEC2BF009C
:105AF0000080FB004300DE000080FB0061006000CE
:105B00000000E0005B003A003408E2005900320077
:105B100040498000E20F500038003A0030498000D0
:105B2000E20F500004003A00014D8000C0F6210051
:105B3000AE0B070003003700014D8000108F2100DD
:105B4000AA0B0700803E200060678800CEC2BF001D
:105B50000080FB004300DE000080FB00610060006D
:105B60000000E00008003A00EC0CE200F7FF3A0009
:105B7000014D8000A00020000088B900800078005E
:105B8000C0F62100990B0700EC0CE20012003A006D
:105B900032458000434580005245880063458800B7
:105BA000534980006349880000C4B30026040700FD
:105BB000D0E82D00E4050700CEC2BF000080FB0046
:105BC0004300DE000080FB00610060000000E00098
:105BD000F9FF32001E003700304980000000E80065
:105BE0003049880030498000E20F5000180034002E
:105BF0000000EB0030498800150037004049800064
:105C00008000E90030498000810F500004003A0014
:105C1000014D8000C0F62100740B0700030037001F
:105C2000014D8000108F2100700B0700304980006B
:105C30000000E80030498800314980004049800078
:105C4000808F5000020035000000EB0030498800D2
:105C50004006200087080700CEC2BF000080FB007E
:105C60004300DE000080FB00610060000000E000F7
:105C7000F9FF3200CEC2BF000080FB004200DE0010
:105C80000080FB00610060000000E0002B003A0093
:105C90003408E20029003200104180000000D000EA
:105CA000A49220000400400031002000908F1000DA
:105CB00004003A00014D8000C0F621004B0B0700A4
:105CC00003003700014D8000108F2100470B0700B3
:105CD000104180000000D000A2922000020040008D
:105CE0001008E800104180000000D000A3922000BE
:105CF0000300400034002000900F12000600340022
:105D0000104180000000D000A292200082004000DC
:105D10000000EB00800878004006200055080700CE
:105D2000CEC2BF000080FB004200DE000080FB000E
:105D3000610060000000E000F9FF3200CEC2BF0049
:105D40000080FB000000D1000080FB0061006000CB
:105D50000000E00020003A006E09E20004003A0072
:105D6000014D8000C0F62100200B07000A0037001B
:105D7000704B8000E20F500004003A00014D80009B
:105D8000108F2100190B070003003700014D800020
:105D9000904F2100150B0700704B80000000E900B8
:105DA000704B88006E09E20002003D0020002000D8
:105DB000704B8800400620002E080700CEC2BF00AE
:105DC0000080FB000000D1000080FB00610060004B
:105DD0000000E000F9FF32000040EB009A030700EA
:105DE00023438000131798001E129000E10F520009
:105DF000220132001E109000E10F50000300340019
:105E00009E109000E28F5000120332003DFA07000E
:105E100032438000620F9800EE099000E28F51003B
:105E20004F0032006E0A9000E20F520007003C0063
:105E30006E0890000000E0000A003200EE089000BA
:105E4000E18F500044003200060037006E099000D8
:105E5000E30F510052003200EE099000E48F510030
:105E600086003200104180000000D000A492200083
:105E7000040040001000E00004003A0070C0B300CD
:105E8000A3030700E0E92D002F0507001041800063
:105E90000000D000A192200001004000120020006C
:105EA000900F110004003A0070C0B300980307007F
:105EB00020EA2D0024050700104180000000D000DA
:105EC000A39220000300400024002000900F120045
:105ED00004003A0070C0B3008D03070060EA2D0093
:105EE00019050700104180000000D000A192200099
:105EF0000100400032002000900F110002003A0023
:105F0000A0EA2D00100507003408E20003003A0063
:105F1000F0EA2D000C050700590037006E09E20079
:105F200002003A0040EB2D0007050700704B80008F
:105F3000E10F500002003A0090EB2D00020507002F
:105F4000704B8000E20F50004D003A00E0EB2D0056
:105F5000FD0407004A003700F2F907004800370047
:105F60003408E2000B003A0030EC2D00F604070084
:105F70009808E20003003A0070EC2D00F2040700DC
:105F80003F00370021002000C044800027060700A2
:105F90003B003700D0EC2D00EB0407003800370041
:105FA000A000200085070700CF80DE00924380001C
:105FB000A34380000201400083814800924388008F
:105FC000A3438800E06980000000E800E0698800E1
:105FD000E0698000EF0F5000290034000000EB0062
:105FE000E069880090438000A1438000CC09DD0077
:105FF0004400DE0000807100C488DE00824C800016
:106000000202B800924C80000283B90005017800BA
:1060100006014100834C80000198B9000001410055
:1060200082027800340F9800450F98006000B80095
:1060300090438800A14388003E089000CE0890005D
:10604000480ADD004800DE0000007200C808DE00DB
:106050008043880070C0B3002D03070060ED2D0061
:10606000B90407002100200080438000EF050700ED
:1060700080ED2D00B404070001003700DAF90700B5
:1060800000C4B300F00207000E08E20024003A004A
:106090002A812000F0408000014180004F8ADE000C
:1060A000CFA2DE00F04080000141800004017800B2
:1060B00084017800444C8000554C80004FACDE00D9
:1060C000CFC4DE00444C8000554C800008037800AB
:1060D00088037800DBF30700009DBE000295BE0038
:1060E000208120005001BE004000BE0014022000AC
:1060F0008381D1000281D3008180D3000080D3004E
:106100000402E900FAFF3A00300F9800410F9800AE
:106110003E089000CE089000800507000A00370076
:10612000F040800001418000809FBE00A0ED2D0066
:10613000801F7800C083200081E80700E6875700B1
:10614000C0832000800407006C08E20048003A0089
:10615000304B8000E10F500027003A00A041800042
:10616000E10F500024003A002A81200020418000E5
:10617000314180004F8ADE00CFA2DE002041800046
:10618000314180000401780084017800444C800093
:10619000554C80004FACDE00CFC4DE00444C800084
:1061A000554C80000803780088037800A5F30700A9
:1061B000009DBE000295BE00208120005001BE005F
:1061C0004000BE00140220008381D1000281D30070
:1061D0008180D3000080D3000402E900FAFF3A0076
:1061E00020079800F0ED2D00570407002E009000C6
:1061F000510507003702370030498000E20F500098
:1062000006003A0040498000E20F500003003A00C7
:1062100020EE2D004C0407000500370080EE2D0015
:1062200049040700304980001004B0001F04070033
:1062300020498000E10F500002003A00D0EE2D000E
:106240004104070020498000E20F500002003A009C
:1062500000EF2D003C04070020498000E40F5000AF
:106260001C023A0030EF2D003704070019023700F6
:1062700060EF2D0034040700160237000040EB00E9
:10628000710207001FF9070070C0B300A0020700E9
:10629000E0EF2D002C04070000C4B3006A020700E1
:1062A000404380006101B900720F98000317980005
:1062B000C0002000010020007E0990008E11900097
:1062C000800F5100818F590010003E007E08900021
:1062D0008E109000006001000C0037001D00370098
:1062E000710037008200370093003700A4003700A8
:1062F000C70037001E0137002F0137004A01370061
:106300006501370088013700AA01370079070700C7
:10631000000F78001E00E000020034001000200092
:10632000404B88001E00E00002003D000000EB0032
:10633000404B88006809E2000300320060F02D0045
:1063400001040700E301370070F12D00FE03070090
:10635000E0013700704B80000000D0004197200022
:1063600081044000704B80000000D0004297200064
:1063700002044000A000200068070700980C1000ED
:10638000704B80000000D0004397200003014000C4
:1063900081BA2D00704B80000000D0000100400049
:1063A00012017800900F510009003D00704B8000F1
:1063B0000000D000449720000401400081BA2D0065
:1063C000704B80000000D0000100400010097800F0
:1063D000704B80000000D000419720000101400078
:1063E000E1BA2D00704B80000000D0000100400099
:1063F00012017800900F510009003400704B8000AA
:106400000000D0004397200003014000E1BA2D00B6
:10641000704B80000000D00001004000100978009F
:106420006E09E20002003A0080F22D00C603070068
:10643000704B8000E10F500002003A00C0F22D00C6
:10644000C1030700704B8000E20F500002003A00C9
:1064500000F32D00BC03070040F32D00BA03070032
:10646000704B80000000D0004497200004004000E2
:10647000100078006101B900804F22001100200057
:10648000C0F20700809FBE00B0F32D00801F78008F
:10649000C0832000AAE70700E6875700C0832000DA
:1064A000A90307008B01370012070700000F7800CF
:1064B0001E00E0000200340010002000504B880055
:1064C0001E00E00002003D000000EB00504B880081
:1064D0006A09E2000300320040F42D009A0307002D
:1064E0007C01370050F52D00970307007901370034
:1064F00000070700000F78001E00E00002003400D3
:1065000010002000604B88001E00E00002003D00EB
:106510000000EB00604B88006C09E20003003200D1
:1065200060F62D00880307006A01370070F72D0020
:106530008503070067013700EE060700000F7800AB
:106540001E00E0000200340010002000004C880013
:106550001E00E00002003D000000EB00004C88003F
:106560008009E20003003A0080F82D00760307005E
:106570005801370090F92D007303070055013700CB
:10658000A0002000E5060700E14B800000804000ED
:10659000E04B88007C09E20002003D000000EB00B7
:1065A000E04B8800E04B8000E30F50000200340015
:1065B00030002000E04B8800A0FA2D0062030700A5
:1065C0007C09E20002003A0030FB2D005E03070068
:1065D000E04B8000E10F500002003A00C0FB2D00AC
:1065E00059030700E04B8000E20F500002003A0020
:1065F00050FC2D0054030700E04B8000E30F5000D7
:1066000034013A00E0FC2D004F0307003101370050
:10661000B8060700CF80DE0003AF2D001302B800DC
:10662000130190000283B9000501780006014100C2
:10663000930178000198B9000001410082027800BE
:10664000F0488000014980000000420081804A003B
:10665000F048880001498800F24880000349800022
:10666000F0D02C0001002000800F5100818F5900D4
:1066700004003400F0D02C0001002000F048880015
:1066800001498800F248800003498000C07E230051
:1066900001002000800F5100818F590004003C0050
:1066A000D07E230001002000F048880001498800C6
:1066B0002A812000F0488000014980004F8ADE00D6
:1066C000CFA2DE00F048800001498000040178007C
:1066D00084017800444C8000554C80004FACDE00B3
:1066E000CFC4DE00444C8000554C80000803780085
:1066F0008803780053F20700009DBE000295BE009B
:10670000208120005001BE004000BE001402200085
:106710008381D1000281D3008180D3000080D30027
:106720000402E900FAFF3A00200798002E009000CA
:106730000000D0006101B900000E270021072000F1
:1067400065F20700104988002E009000801F780035
:1067500070FD2D00801F7800C0832000F8E6070040
:10676000E4875700C0832000F7020700D9003700F4
:1067700060060700000F78001E00E00002003400F1
:1067800010002000104C88001E00E00002003D00B8
:106790000000EB00104C88008209E2000300320088
:1067A00080FE2D00E8020700CA00370090FF2D0090
:1067B000E5020700C70037004E060700800078009A
:1067C000A00020000088B900924B8000000041002A
:1067D000904B8800914B8000C0442000808F500077
:1067E00002003400C0442000904B88007209E2008F
:1067F00002003D000000EB00904B88007209F80099
:10680000A0002E00801F7800C0832000CCE6070087
:10681000E4875700C0832000CB020700904B800024
:10682000EC070700AB003700320607008000780055
:10683000A00020000088B900824B800000004100C9
:10684000804B8800814B8000C0DA2000808F500090
:1068500002003400C0DA2000804B88007009E2009A
:1068600002003D000000EB00804B88007009F8003A
:10687000C0012E00801F7800C0832000B0E6070012
:10688000E4875700C0832000AF020700804B8000E0
:10689000D60707008F003700A00020001F06070062
:1068A000F14B800000804000F04B88007E09E20040
:1068B00002003D000000EB00F04B8800F04B800030
:1068C000E30F50000200340030002000F04B88003D
:1068D000C0022E009C0207007E09E20002003A007E
:1068E00050032E0098020700F04B8000E10F50008B
:1068F00002003A00E0032E0093020700F04B8000F4
:10690000E20F500002003A0070042E008E020700D1
:10691000F04B8000E30F50006E003A0000052E009F
:10692000890207006B003700A0002000FB0507006C
:10693000500F98005E0890000000E0000F00320049
:10694000204C8000DE08900001004000204C8800B0
:106950008409E20002003D000000EB00204C8800AA
:10696000204C8000E70F500002003400700020002F
:10697000204C8800204C80003A040700214C800005
:10698000800020000008B80082B62D000000410001
:10699000801F780090052E00801F7800C0832000A3
:1069A00067E60700E4875700C083200066020700FF
:1069B00048003700A0002000D805070080007800BC
:1069C0004049800001004000404988004049800063
:1069D000E10F500002003C002000200040498800E8
:1069E00040498000FA0F500002003400A00120004E
:1069F000404988003149800040498000808F500024
:106A00000200340043498000334988004049800037
:106A1000E20F500006003A0060062E00801F78004A
:106A2000C083200046E607008F87E9000600370094
:106A30002809F80070072E00801F7800C08320000E
:106A40003FE60700E4875700C08320003E020700AE
:106A5000200037000040EB007B000700F04380007F
:106A60000144800002BA2B00D300200045F107004A
:106A7000801F78007808F80090082E00801F7800AA
:106A8000C08320002EE60700E6875700C083200061
:106A90002D02070000C4B3006B0007001044800003
:106AA0002144800002BA2B00D300200035F10700FA
:106AB000801F78007A08F80040092E00801F7800B7
:106AC000C08320001EE60700E6875700C083200031
:106AD0001D020700F44B8000241798002E10900030
:106AE000E10F500014003200AE109000E18F500012
:106AF00004003C002E1190000200E000050032006E
:106B000011003700AE119000E28F51000C003200EE
:106B10000D003700F10307000000E0000B00320019
:106B2000FE030700F0092E00801F780023E607000F
:106B30008F87E90005003700AD0D0700030037001F
:106B4000DA10070001003700C30A07000C12070023
:106B5000CFC2BF000080FB004600DE000080FB00CB
:106B600061006000E10F500099F93A000FF807004A
:106B700097F937000200FA00004F78000900FC0086
:106B8000B1168000F00F2000008160001E80FB0025
:106B9000C800DD0000F02F000080600000007100E0
:106BA000B01688001000200095040700D6A2A800A7
:106BB0001000200092040700D6A2A90010002000B7
:106BC0008F0407000080FA00000006000200FA00AF
:106BD00000002800000F78000400FC0091168000DF
:106BE00000F02F000080700090168800D6C2A80028
:106BF000D6E2A9001E00E0000A003D0010002000BF
:106C00007F040700D6A2A800200020007C04070013
:106C1000A116800000F02F00008F6000D6A2A9000E
:106C2000F4FF3700D6C2A900D6E2A8000400FC0099
:106C300090168000F10F200001006000901688007F
:106C40000080FA00000006000200FA00004F780001
:106C5000DEFF0700D6E2A90000C8B3001E407000A6
:106C6000C4FF0700D6E2A8000080FA00000006007A
:106C70000000FA00D5FF0700D6E2A90010C0B3005B
:106C8000BCFF0700D6E2A8000080FA000000060062
:106C90000000FA00D6E2A900D6C2A900F000200048
:106CA0007404070080C3B300B2FF07005000200047
:106CB0007004070080C3B300AEFF0700100020007F
:106CC0006C04070080C3B300AAFF07001000200077
:106CD00068040700C0C0B300A6FF07001000200032
:106CE0006404070010C0B300A2FF070020002000CA
:106CF0006004070060C0B3009EFF07001000200082
:106D00005C040700D6E2A8000080FA00000006003C
:106D10000200FA00004F7800ACFF07001E40780028
:106D200094FF07000080FA00000006000200FA004D
:106D3000004F780011479800A4FF0700D6E2A90091
:106D4000F0C3B3001E4F600000C4B3001E407000CB
:106D500088FF0700D6E2A8009CFF07001E409000B5
:106D600084FF0700C2FF07000080FA000000060051
:106D70000400FA00004F7800114798000040EB0033
:106D800020479800AE4090001E40900080CF5000F9
:106D900007003D008DFF07001E40780075FF0700CB
:106DA0002E4090000040E80020479800F5FF370093
:106DB0000080FA00000006000000FA0083FF0700D0
:106DC000D6E2A90000C4B3006AFF0700D6E2A8001B
:106DD00011C0B3000040EB00E5FF070051C0B30055
:106DE00000C1B300E2FF070021C0B3000040EB0088
:106DF000DFFF070011C0B3000040EB00DCFF07001D
:106E000051C0B30040C1B300D9FF070021C0B30097
:106E10000040EB00D6FF070011C0B3000040EB00BC
:106E2000D3FF070051C0B30050C1B300D0FF07002B
:106E300021C0B3000040EB00CDFF070011C0B3003C
:106E40000040EB00CAFF070051C0B30010C0B30000
:106E5000C7FF070021C0B3000040EB00C4FF0700DC
:106E600011C0B3000040EB00C1FF070051C0B300E8
:106E700050C0B300BEFF070021C0B3000040EB00CC
:106E8000BBFF070021C0B3000040EB00B8FF0700C4
:106E900011C0B30000C1B300B5FF070011C0B300BB
:106EA0000040EB00B2FF070011C0B30000C1B30007
:106EB000AFFF070031C0B3000040EB00ACFF07009C
:106EC00031C0B3000040EB00A9FF070011C0B300C0
:106ED00000C1B300A6FF070041C0B3000040EB00B3
:106EE000A3FF070021C0B3000040EB00A0FF070094
:106EF00031C0B30000C1B3009DFF070031C0B30033
:106F00000040EB009AFF070059FF07000080FA00DD
:106F1000000006001200FA00000F780000032000B5
:106F20009E0F10000200340000032000000F7800C4
:106F30001E00780062002000110009000200D80045
:106F4000200798001E007800620020001100090050
:106F50000200D8008000FD00300798000000EB0020
:106F6000400798000000EB00100798001E009000FA
:106F7000E70F50000E003C00EA0047004E00900072
:106F800000814000E10C2E001E00900000804000B7
:106F9000104978004E0090000000E800400798007B
:106FA0001E0090000000E80010079800EFFF370077
:106FB0000000EB00400798002E0090000000E00069
:106FC0000C003400EA0047004E0090008080400032
:106FD00020C0B300804878004E0090000000E80018
:106FE000400798002E0090000000E900200798005C
:106FF000F1FF37003E0090000000E0000700340081
:10700000EA0047004E00900000814000210C2E0055
:107010003E00900000804000104978000000EB0026
:10702000100798001E009000E70F500009003C0078
:10703000EA0047001E0090000080400010407800E9
:1070400033FF07001E0090000000E80010079800C2
:10705000F4FF37000080FA00000006001600FA0076
:10706000000F780011079800000320009E0F100009
:107070000200340000032000000F78008000200090
:10708000500798001E0078006200200011000900DF
:107090000200D800300798001E007800620020002F
:1070A000110009000200D8008000FD004007980090
:1070B0001E0090000000E00036003A000000EB00E7
:1070C000600798003E0090000000E0000F003400D0
:1070D000EE0047006E0090008080400020C0B300AA
:1070E000804878006E0090000000E800600798007B
:1070F0003E0090000000E900300798005E0090001C
:107100000000E90050079800EEFF37004E009000A5
:107110000000E0000D003400EE0047006E0090001B
:1071200000814000210C2E004E00900000804000A5
:10713000104978006E0090000000E8006007980099
:107140005E0090000000E900500798000000EB008E
:1071500020079800AE0090005E009000808F5000E5
:1071600042003D00EE0047006E009000808040002D
:1071700000C2B300804878006E0090000000E80074
:10718000600798002E0090000000E800200798009B
:10719000F0FF370070002000600798003E0090006C
:1071A0000000E0000F003400EE0047006E00900089
:1071B0008080400020C0B300804878006E009000BE
:1071C0000000E900600798003E0090000000E90020
:1071D000300798005E0090000000E900500798001A
:1071E000EEFF37004E0090000000E0000D0034007C
:1071F000EE0047006E00900000814000810C2E00E0
:107200004E00900000804000104978006E00900011
:107210000000E900600798005E0090000000E900AF
:10722000500798000000EB0020079800AE00900087
:107230005E009000808F50000C003D00EE00470083
:107240006E0090008080400000C2B300804878004B
:107250006E0090000000E900600798002E0090008A
:107260000000E80020079800F0FF37000000EB0066
:10727000200798002E009000E70F500009003C0006
:10728000EE0047002E009000008040001040780083
:107290009FFE07002E0090000000E80020079800E5
:1072A000F4FF37000080FA00000006000200FA0038
:1072B000004F78001E40780095FE07000080FA001D
:1072C000000006000200FA00004F78001E4078001F
:1072D000104798001E80FB004400DE00004F78003D
:1072E00090C0B3009E4F100003003E0000C3B300E7
:1072F0001E4F40000200370070C3B3001E4F400015
:107300001E40780082FE07001E409000004F78006B
:107310001E4078006F4F600090C0B3009E4F100079
:1073200003003E0000C3B3001E4F400002003700C0
:1073300070C3B3001E4F40001E40780074FE07006B
:107340000080FA00000006000200FA00000F78003A
:107350001E0078001004E000070032009E00780054
:10736000114078006AFE07001E0078000000E80067
:10737000000F7800F6FF37000080FA0000000600DA
:107380000600FA00008FBE00424798004E40900071
:107390000004E0002E003A001E00BE0002A02C00F7
:1073A000A3B92300F7EE07000043B00058FE070022
:1073B0001E00BE0002A02C00A3B92300F1EE0700BE
:1073C00002A02C000202B800A2B923000283B90077
:1073D000050178000601410003A02C000388B900D4
:1073E00000014100820278001E1F12001E971A0041
:1073F000E0C2B30046FE07001E00BE0002102E00D1
:10740000535F2000DFEE07000043B00040FE07009E
:107410001E00BE0002102E00535F2000D9EE0700B0
:1074200002102E000202B800525F20000283B90051
:10743000050178000601410003102E000388B90001
:1074400000014100820278001E1F12001E971A00E0
:107450004E4090000004E0000A0032001E00BE0012
:107460000268290083092000C6EE0700E00F5000E3
:10747000E08F580003003A0000C2B30024FE07006A
:10748000060037001E00BE000268290083092000A4
:10749000BCEE07000043B0001DFE07001E00BE004A
:1074A0000268290083092000B6EE0700026829005F
:1074B0000202B800820920000283B90005017800A9
:1074C00006014100036829000388B900000141005A
:1074D000820278001E1F12001E971A001E00BE00B6
:1074E00002242400F3002000A6EE07000043B000B1
:1074F00007FE07001E00BE0002242400F300200047
:10750000A0EE0700022424000202B800F2002000CE
:107510000283B9000501780006014100032424001C
:107520000388B90000014100820278001E1F12008A
:107530001E971A00E0C2B300F5FD07001E00BE0052
:10754000026A2800130020008EEE07000043B000FE
:10755000EFFD07001E00BE00026A28001300200095
:1075600088EE0700026A28000202B800120020001C
:107570000283B9000501780006014100036A280072
:107580000388B90000014100820278001E1F12002A
:107590001E971A001E00BE00027122000300200088
:1075A00078EE07000043B000D9FD07001E00BE00C2
:1075B000027122000300200072EE07000271220017
:1075C0000202B8000001EB000283B9000501780057
:1075D00006014100037122000388B9000001410047
:1075E000820278001E1F12001E971A001E00BE00A5
:1075F000823E20000300200062EE07000043B0003E
:10760000C3FD07001E00BE00823E200003002000D4
:107610005CEE0700823E20000202B8000001EB0091
:107620000283B9000501780006014100833E200075
:107630000388B90000014100820278001E1F120079
:107640001E971A00E0C2B300B1FD07001E00BE0085
:1076500042062000030020004AEE07000043B0006D
:10766000ABFD07001E00BE00420620000300200004
:1076700044EE0700420620000202B8000001EB00C1
:107680000283B9000501780006014100430620008D
:107690000388B90000014100820278001E1F120019
:1076A0001E971A001E00BE00A2002000030020004A
:1076B00034EE07000043B00095FD07001E00BE0039
:1076C000A2002000030020002EEE0700A2002000F0
:1076D0000202B8000001EB000283B9000501780046
:1076E00006014100A30020000388B9000001410009
:1076F000820278001E1F12001E971A004E40900052
:107700000004E00003003A0001C3B3001EC04000C3
:107710007FFD07000080FA00000006000400FA0068
:10772000008FBE0012C0B3001E00BE0014FF070091
:107730000080FA00000006000200FA00000F780046
:107740001E00E00002003400B0C2B30070FD07006C
:107750001E00E00002003A0000C2B3006CFD07000A
:107760001E00E00003003D00D0C2B30068FD07002A
:107770001E0FEA001E007800823E20001100090062
:107780000200D8000043B00061FD07001E00780031
:10779000823E2000110009000200D8008000FD0098
:1077A000803E20000088B9001E0F1000E0C2B30028
:1077B00057FD07001E007800420620001100090056
:1077C0000200D8000043B00051FD07001E00780001
:1077D00042062000110009000200D8008000FD00D0
:1077E000400620000088B9001E0F10001E0078001F
:1077F000A2002000110009000200D8000043B000E0
:1078000043FD07001E007800A200200011000900BF
:107810000200D8008000FD00A00020000088B90010
:107820001E0F10000080FA00000006000400FA009D
:10783000000F780011079800F07022009E0F1000D2
:1078400002003400F0702200000F78001E00780063
:10785000823E2000110009000200D8000000E00074
:107860000F0032001E007800823E20001100090047
:107870000200D8000043B00025FD07001E0078007C
:10788000823E2000110009000200D8008000FD00A7
:10789000803E20000088B9001E0F10000200370053
:1078A00000C2B3001AFD07001E0078004206200047
:1078B000110009000200D8000043B00014FD0700C9
:1078C0001E00780042062000110009000200D800C6
:1078D0008000FD00400620000088B9001E0F100047
:1078E0001E009000E20F5000040032009E00900045
:1078F00070072000808F500002003A00E0C2B30001
:1079000003FD07001E007800A200200011000900FE
:107910000200D8000043B000FDFC07001E00780004
:10792000A2002000110009000200D8008000FD0024
:10793000A00020000088B9001E0F10001E0090005B
:10794000E10F500002003A00E0C2B300F0FC070073
:107950009E00900070072000808F500003003A00C6
:1079600070C5B300EAFC07000300370001C3B30091
:107970001EC04000E6FC07000080FA000000060080
:107980000200FA00004F780090C0B3009E4F100034
:107990000200340090C0B300004F780001C3B30070
:1079A0001EC04000DAFC07000080FA00000006005C
:1079B000809FBE000200FA0090108000004F780007
:1079C0003ECDBF000080FB008000E800B6C9BF00CC
:1079D0000080FB00808F5000080032003ECDBF00C9
:1079E0000080FB00719B2000010040001E487800D1
:1079F0003ECDBF000040E8003EEDB7000EC2BF0024
:107A00000080FB000000D1000080FB0061006000EE
:107A1000E10F500001003A000E22A9008520A900C4
:107A20000080FA004F00BE00004006000000FA008F
:107A3000600D2E0030009000A01088000000EB00C8
:107A4000601088000000EB00701088000F42A80052
:107A50008520A9008D20A8000DE2A8000080FA0072
:107A6000000006000200FA00000F780070002000FD
:107A70009E0F10000200340070002000000F7800FC
:107A8000610D2E001E0078000000D00001004000B3
:107A900010007800A01088000080FA0000000600A6
:107AA0000200FA00004F78000FC2BF000080FB0008
:107AB0000000D1000080FB0061006000E10F500079
:107AC000F9FF32001E00FB00F10F200001006000F2
:107AD000801088000080FA00000006000200FA0012
:107AE000E1D3200091407800B6C9BF0000C050002B
:107AF000004FE9001E80FB000080FA000000060035
:107B00000000FA000040EB00B6E9B70010C0B30077
:107B10003EEDB7000080FA00000006000000FA0009
:107B200000000000B6C9BF000080FB008000E80034
:107B30003ECDBF000080FB00808F5000F9FF320077
:107B4000B6C9BF000040E800B6E9B7000080FB00FE
:107B5000719B2000010040001080FB000080FA00B3
:107B6000000006000200FA00ECFF0700004F78005A
:107B70001E407800CAFF07001E80FB000080FA004C
:107B8000000006000600FA006000B800008FBE008A
:107B9000E2FF07000074A100404798004E409000AB
:107BA000BFFF0700CE409000F0C2B30080CF50006E
:107BB00016003400CE40900090C3B30080CF500038
:107BC00012003C001E00BE00A20020000203B8000C
:107BD0000001EB000282B9000701780004014100B6
:107BE000A30020000388B90000014100820378004F
:107BF0004E4090000000FB0001FD2F0001004000FE
:107C0000CF80DE00001F430001974B004E409000E4
:107C1000ED4F5000DEFF3A001E00BE000080FA006B
:107C2000000006000600FA00881F7800008FBE00E2
:107C300090C0B300504798000040EB0040479800C8
:107C40004E409000E94F500016003C005E4090000E
:107C50000000FB0071AB2000010440001E00BE00CC
:107C6000A2002000030020002BED070002C3B30098
:107C7000024C40001E00BE00A200200003002000B5
:107C800015ED0700008FBE005E4090000040E90047
:107C9000504798004E4090000040E8004047980050
:107CA000E7FF37000040EB00C1EAB7004F0478005F
:107CB0000080FA00000006000400FA00008FBE00F9
:107CC0001E00BE00D7FF0700B7CABF0074FF070041
:107CD000B8CABF0072FF0700B9CABF0070FF070033
:107CE000BACABF006EFF0700BBCABF006CFF070027
:107CF000BCCABF006AFF0700BDCABF0068FF07001B
:107D0000BECABF0066FF0700BFCABF0064FF07000E
:107D1000C0CABF0062FF07000080FA000000060032
:107D20000200FA003ECDBF000080FB00801F7800FB
:107D3000B6C9BF000080FB00801F7800600E2E00D7
:107D4000801F78009DE10700E68757000000EB00E8
:107D5000000F7800E00F20009E0F100006003C008E
:107D6000719B20001E804000104078004CFF0700EF
:107D70001E0FE800F7FF37000080FA000000060041
:107D80000000FA000000EB0050158800F01F2000F2
:107D900040158800F0002000301588000008200001
:107DA000201588000000EB00101588000000280056
:107DB000001588000080FA00000006000200FA00AA
:107DC000000F78009E0078006F80600030158800FA
:107DD000A022A800401F200009000700A022A9003F
:107DE000A0C2BF000080FB00610060000000E00056
:107DF000FBFF3200001480000080FA000000060043
:107E00000200FA00000F78000000EB00C0088800B4
:107E10001E00780001002000820020000202B8004D
:107E20000001EB000283B900050178000601410062
:107E3000830020000388B90000014100820278001D
:107E4000E408880086C0A90021E1A80086C0BF0020
:107E50000080FB004600DE000080FB006100600047
:107E60000000E000F9FF320021E1A9000080FA00E3
:107E7000000006000400FA00000F78000000EB008C
:107E8000100798001E0090009E0F50000600310061
:107E9000803E2000DAFF07001E0090000000E8008E
:107EA00010079800F7FF37000080FA000000060076
:107EB000809FBE00821F78000200FA000000EB00E5
:107EC000000F780082C0BF000080FB004400DE008D
:107ED0000080FB00610060000000E00002003A004A
:107EE00011002000010F78009E40780061C0600002
:107EF0004401DD002108200091407800F0CEB3005D
:107F000000C060000240700082E0B70088A0A900B5
:107F100010C0B3001AEDB7001C0DE20024003200BF
:107F200082C0BF000080FB004400DE000080FB0038
:107F3000610060000000E0000F003A00C3C2BF0013
:107F40000080FB004600DE000080FB006100600056
:107F50000000E00004003200C06880000000E8007B
:107F6000C068880012003700C06880000000E90087
:107F7000C06888000E003700C3C2BF000080FB004D
:107F80004600DE000080FB00610060000000E000B1
:107F900004003200C06880000000E900C06888006A
:107FA00003003700C06880000000E800C068880057
:107FB0000000EB00E06888000080FA004F017800C4
:107FC0004F00BE0000400600809FBE00821F780068
:107FD0000200FA000000EB00000F780082C0BF0032
:107FE0000080FB004300DE000080FB0061006000B9
:107FF0000000E00002003A0011002000010F7800AC
:108000009E40780061C060004301DD00210820002F
:108010009140780070CFB30000C060000240700053
:1080200082E0B7008880A90010C0B3001AEDB70045
:108030001C0DE20022003A0082C0BF000080FB005D
:108040004300DE000080FB00610060000000E000F3
:108050000E003A00C3C2BF000080FB004700DE00F4
:108060000080FB000000E00004003200C0688000D7
:108070000000E900C068880011003700C068800077
:108080000000E800C06888000D003700C3C2BF00D0
:108090000080FB004700DE000080FB000000E000E5
:1080A00004003200C06880000000E800C06888005A
:1080B00003003700C06880000000E900C068880045
:1080C00010002000E06888000080FA004F0178006E
:1080D0004F00BE00004006000000FA0088A0A90082
:1080E00090A0A8008880A9009080A8000080FA00D5
:1080F000000006000200FA00C0688000000F78004F
:108100000000EB00C06888000040EB001AEDB700EB
:108110001E0078000080FA00000006000600FA0049
:10812000000F7800C06880009E0F500007003400E8
:108130000000EB00C06888000040EB001AEDB700BB
:1081400010002000200798000D0037009E00EA0074
:10815000C0688000810F500007003D000000EB0068
:10816000C06888000040EB001AEDB7000080EB000B
:1081700020079800020037000000EB00200798005D
:108180002E0090000080FA00000006000200FA00B5
:10819000004F78000040EB00104798001E40900010
:1081A000E74F500010003C001E80FB0061006000A3
:1081B0000000E00002003200E202A80001003700E7
:1081C000E202A900E222A8001E80FB000000D1000C
:1081D000004F7800E222A9001E4090000040E80015
:1081E00010479800EDFF37000080FA0000000600FD
:1081F0000600FA00008FBE001E00BE00F068880076
:10820000016988000040EB00404798004E40900014
:10821000E44F50000A003C004E4090000000FB007C
:10822000E1D120000100400010407800D7FF070096
:108230004E4090000040E80040479800F3FF3700B0
:10824000E822A800E822A9000080FA000000060049
:108250000000FA00E802A800E202A900E802A90072
:10826000E822A800E822A90010C0B30022EDB70060
:108270000080FA00000006003200F800900188003B
:108280006118E100040032007018E10002003200C1
:10829000F0FF2F00030037003119BA008301E90015
:1082A000FDFF3A003200F90000000600849FBE0086
:1082B0004220A900440424006110E1000A003200B9
:1082C000540424007010E10007003200640424000C
:1082D000F5FF2F000510E10003003200F0FF2F0032
:1082E0004F02BE00000006003200F800203B88006C
:1082F000113B8800043B88000500FC00500520006D
:10830000303B8800A00A2000303B880061E7A800CD
:10831000000000000000000061E7AF00FEFF370032
:108320000000EB003200F9004F02BE000000060022
:10833000841F78004220A900440024006118E10055
:1083400006003200540024007018E10003003200DF
:108350004F027800F0FF2F00000006003200F80006
:1083600091018800821F78003019BB008301E90069
:10837000FDFF3A00213B88004F017800123B880046
:10838000043B88000500FC0050052000303B8800BD
:10839000A00A2000303B880061E7A8000000000030
:1083A0000000000061E7AF00FEFF37000000EB00B7
:1083B0003200F9004F027800000006003600F80095
:1083C000809FBE00829FBE00849FBE00869FBE002D
:1083D0000200FA0030032000A01088000000EB002B
:1083E000000F7800F0CF27009E0F100003003C0024
:1083F000000000001E0FE800FAFF370020102E00DA
:10840000801F7800EDDF07008F87E9004207F80042
:10841000C0112E00801F7800E8DF0700E4875700B6
:108420009A000700FFFF37003600F800809FBE006B
:10843000829FBE00849FBE00869FBE000000FA009F
:10844000B0658800C1658800D2658800E365880052
:10845000F46588000566880016668800276688002F
:1084600038668800496688005A6688006B6688000E
:108470007C6688008D6688009E668800AF668800EE
:10848000A0122E00801F7800CCDF07008F87E90044
:10849000B60CF80020142E00801F7800C7DF0700FC
:1084A000E4875700B80CF800C0142E00801F780035
:1084B000C2DF0700E4875700BA0CF80060152E00F1
:1084C000801F7800BDDF0700E4875700BC0CF80070
:1084D00000162E00801F7800B8DF0700E4875700E1
:1084E000BE0CF800A0162E00801F7800B3DF070036
:1084F000E4875700C00CF80040172E00801F78005A
:10850000AEDF0700E4875700C20CF800E0172E002A
:10851000801F7800A9DF0700E4875700C40CF8002B
:1085200080182E00801F7800A4DF0700E487570022
:10853000C60CF80020192E00801F78009FDF07006E
:10854000E4875700C80CF800C0192E00801F78007F
:108550009ADF0700E4875700CA0CF800601A2E0063
:10856000801F780095DF0700E4875700CC0CF800E7
:10857000101B2E00801F780090DF0700E487570053
:10858000CE0CF800C01B2E00801F78008BDF070088
:10859000E4875700D00CF800701C2E00801F780074
:1085A00086DF0700E4875700D20CF800201D2E005C
:1085B000801F780081DF0700E4875700D40CF800A3
:1085C000D01D2E00801F78007CDF0700E487570055
:1085D0002E000700FFFF37003600F800809FBE0026
:1085E000829FBE00849FBE00869FBE000000FA00EE
:1085F000AF6688000F902000801E2E00801F78003C
:108600006EDF07008F87E900D40CF800D01D2E0024
:10861000801F780069DF0700E48757001B00070010
:10862000FFFF37003600F800809FBE00829FBE002B
:10863000849FBE00869FBE000000FA00E01F2E004F
:10864000801F78005DDF07008F87E9000F000700BB
:10865000FFFF37003600F800809FBE00829FBE00FB
:10866000849FBE00869FBE000000FA0090A0A90073
:108670009120A90030212E00801F78004FDF0700D5
:108680008F87E90001000700FFFF37000000FA00B4
:1086900077F9070000232E002BFB0700CFC2BF0095
:1086A0000080FB004600DE000080FB0061006000EF
:1086B000E10F5000F9FF3A00CFA2A900F7FF370001
:1086C0000000FA0010002000106788001000200051
:1086D00020678800803E2000B06688000000EB0024
:1086E000800C88000000EB00B00C880040062000E1
:1086F000600C880040062000700C8800E00020001C
:10870000800C8800007D2000900C8800007D2000F7
:10871000A00C8800E0002000B00C8800B0D421003C
:108720007008880013E1A8008CE0A8000080FA001F
:10873000000006000000FA000000EB00200C88009A
:10874000F0002000000C8800F0002000100C8800D1
:1087500060002000200C8800E001200060088800F4
:1087600011E1A8000080FA00000006000000FA00F5
:1087700011E1A9000080FA00000006000000FA00E4
:1087800011E1A8000080FA00000006000000FA00D5
:10879000B06680000080FA00000006000200FA00C7
:1087A000000F7800100020009E0F100002003E0015
:1087B00020002000000F78001E0078000000D1008B
:1087C000000C88001E00E900600888000080FA00A4
:1087D000000006000200FA00000F78001E0078007A
:1087E000600C88000080FA00000006000200FA0019
:1087F000000F78001E007800900C88000080FA00BE
:1088000000000600809FBE00821F78000800FA006A
:10881000F066800030079800BE009000E18F5000A5
:108820000C0032003E009000E10F500006003400C2
:10883000BE009000E28F5000200032003E00900009
:10884000E30F50003B003200D222A8008C60A90048
:108850004C0037008000EB00010F7800D6C2BF004B
:108860000080FB000000D1000080FB006100600080
:108870000000E00002003A0010002000000F780025
:108880009E40780061C060000041D000612D200052
:1088900091407800D0CFB30000C06000024070006B
:1088A000D6E2B700100880000000D1001008880050
:1088B0000000EB00F0668800320037000000EB009B
:1088C00010079800D6C2BF000080FB000000D10056
:1088D0000080FB00610060000000E00002003A0040
:1088E0001100200011079800AE40900061C06000A8
:1088F0000041D000612D200091407800D0CFB3001E
:1089000000C0600002407000D6E2B700D6C2BF00CF
:108910000080FB000000D1000080FB0061006000CF
:108920000000E0001700320010002000F066880010
:10893000140037000000EB0020079800D6C2BF00EB
:108940000080FB000000D1000080FB00610060009F
:108950000000E00002003A0011002000210798000A
:10896000CE40900061C060000041D000612D200029
:1089700091407800D0CFB30000C06000024070008A
:10898000D6E2B7008460A9000080FA004F017800A9
:108990004F00BE00004006000200FA00000F780001
:1089A00030002000F06688001E00E90010088800F2
:1089B000100880000000D10000088800D622A9001D
:1089C000D222A90005E1A8008460A9008C60A8005B
:1089D0000080FA00000006000000FA0020002000DD
:1089E000F06688000080FA00000006000400FA002B
:1089F000000F780011079800DA0CE2000C003A0032
:108A00001E0090000000E00009003400DC0CE200D1
:108A100007003A0059FF0700401F2000104588005A
:108A20001E009000C06688001E007800DAFF070074
:108A30000080FA00000006000000FA000000EB00D1
:108A4000006788003008E20006003200CAE2A80091
:108A500041678000700020000088B90030678800FE
:108A6000CA62A8004167800010498000DFFF07004C
:108A7000406780000000D000D06688000080FA00C7
:108A8000000006000000FA001000200000678800C7
:108A90003008E20006003200CAE2A8004167800008
:108AA000700020000088B90030678800CA62A80002
:108AB00041678000300020000088B9008000780005
:108AC00010498000C9FF0700416780004000200076
:108AD0000088B900D06688000080FA000000060017
:108AE0003600F800809FBE00829FBE00849FBE00BB
:108AF000869FBE000200FA0084E0A900D80CE200C4
:108B00000E003200C06680000000E900C0668800E8
:108B1000D80CE20009003A00AFFF0700304980009E
:108B20000000D000A1922000010040003100200090
:108B3000908F100001003200CA62A900E60CE2002A
:108B400008003200306780000000E90030678800CC
:108B5000E60CE20003003A003008E20001003200B7
:108B6000CAE2A900DA0CE2000C003200D0668000F4
:108B70000000E900D0668800DA0CE20007003A0045
:108B8000E00CE20003003A001000200010678800AB
:108B9000020037001000200020678800EC0CE20083
:108BA00003003200606780000000E9006067880011
:108BB000C0418000E20F500013003A00C8C2BF005D
:108BC0000080FB004500DE000080FB0061006000CB
:108BD0000000E00002003A000000EB00106788008F
:108BE000C8C2BF000080FB004400DE000080FB0024
:108BF000610060000000E0001B003A000000EB0094
:108C00002067880018003700C8C2BF000080FB0042
:108C10004500DE000080FB00610060000000E00015
:108C200003003A000000EB001067880002003700E4
:108C30001000200010678800C8C2BF000080FB0041
:108C40004400DE000080FB00610060000000E000E6
:108C500003003A000000EB002067880002003700A4
:108C60001000200020678800C0418000000F7800BD
:108C70009E007800E28F500004003C001E00780047
:108C80000000E0001A003C00030037009E0078005E
:108C9000E38F500030003200C8C2BF000080FB00EC
:108CA0004500DE000080FB00610060000000E00085
:108CB00004003A00DA0CE20002003A005EFF07000E
:108CC00047003700C8C2BF000080FB004400DE0040
:108CD0000080FB00610060000000E00040003A00FE
:108CE000DA0CE2003E003A0066FF07003C00370065
:108CF000E00CE2000C003200E20CE20004003A005A
:108D0000DA0CE20002003A004BFF070034003700A3
:108D1000E40CE20032003A00DA0CE20030003A00E3
:108D200058FF07002E003700E40CE20004003A0070
:108D3000DA0CE20002003A0052FF07002800370078
:108D4000E20CE20026003A00DA0CE20024003A00CD
:108D500039FF070022003700C8C2BF000080FB00B7
:108D60004500DE000080FB00610060000000E000C4
:108D70000E003A00DC0CE20004003A001000200073
:108D8000E06688001049800003FF07003008E20019
:108D900006003200CAE2A80041678000700020008F
:108DA0000088B90030678800CA62A800C8C2BF0046
:108DB0000080FB004500DE000080FB0061006000D9
:108DC0000000E00006003200DC0CE200040032008B
:108DD000CA62A90000FF07000000EB00E0668800FF
:108DE000B06680000000E900B0668800D60CE200A2
:108DF00005003A00803E2000B0668800B041800047
:108E00000000E800B0418800A208E2000300320040
:108E1000104580000000E90010458800EA0CE200DF
:108E200003003400506780000000E90050678800AC
:108E30000080FA004F03BE004F02BE004F01BE008B
:108E40004F00BE003600F900004006000000FA00A6
:108E5000CA42A9000000EB00306988000000EB0066
:108E6000406988009043200010118800000028000D
:108E7000001188008500A9008D00A8000080FA007C
:108E8000000006000200FA00000F78004069800030
:108E90009E0F10000B00320020C2BF000080FB00BC
:108EA0000000D1000080FB00610060000000E000D5
:108EB000F9FF3A001E007800201188001E0078009B
:108EC000406988000080FA0000000600801F7800DA
:108ED0000200FA00CA42A8008500A90020C2BF0013
:108EE0000080FB00610060000000E0000400320030
:108EF000201180002069880010002000306988005F
:108F0000CA42A9000080FA004F0078000040060025
:108F10001C00FA000000EB003049880030002000FF
:108F2000504988000000EB00000F780050F7070060
:108F300020242E00801F780020DD07008F87E900A5
:108F4000F0252E00801F78001CDD07008F87E900C8
:108F5000C8C2BF000080FB004600DE000080FB00AE
:108F6000610060000000E0000400320010002000FA
:108F7000A0418800CA62A900030037000000EB008E
:108F8000A0418800CA62A800D00020008BFB070027
:108F9000C0438800C000200088FB0700D043880041
:108FA000C1438000C04380000088B900F0438800BE
:108FB00001448800D1438000D04380000088B9007C
:108FC0001044880021448800F2438000034480005C
:108FD000104480002144800000005100818059002D
:108FE000304488004144880034EE0700C3C2BF000B
:108FF0000080FB004500DE000080FB006100600097
:109000000000E00013003A001E0FE800600020009E
:109010009E0F1000020034000000EB00000F7800EB
:1090200021032000E055220070FE0700C3C2BF00EC
:109030000080FB004500DE000080FB006100600056
:109040000000E000F9FF32004006200089FB070025
:1090500028FC07001E017800520F9800DE099000DE
:10906000E38F51009F0032005E089000E30F500034
:1090700007003C005E099000E10F5100270032001C
:10908000DE099000E18F51006F003C0009003700BD
:109090005E089000E50F5000C90032005E099000A4
:1090A000E40F5100AA003400DE099000E68F510061
:1090B000DE0032000040EB00E3F60700C0282E007F
:1090C000A1F8070000C4B300DFF6070009FC0700A1
:1090D000CF80DE00424C8000534C800002014000F3
:1090E00083814800424C8800534C8800E6004700CA
:1090F000424C8000534C8000829FBE00D0292E003D
:10910000801F7800010078008DDC0700E68757009B
:10911000660047008CF80700CC0037000040EB00E9
:10912000C9F60700A000200024FB0700CF80DE0066
:10913000824C80000202B800924C80000283B90089
:109140000501780006014100834C80000198B900B8
:10915000000141008202780014079800250798005A
:109160001E009000AE009000C809DD004800DE003F
:1091700000807100C808DE0080438800802A2E002D
:1091800071F807002100200080438000A7F9070044
:10919000102B2E006CF8070000C4B300AAF60700DD
:1091A00050002000DDFB0700CF80DE00824C8000F5
:1091B000934C80000201400083814800824C88006B
:1091C000934C8800824C8000934C80003006200035
:1091D00001002000800F5100818F590004003C00E5
:1091E0004006200001002000804C8800914C88003F
:1091F000824C8000934C8000800C200001002000F5
:10920000800F5100818F590004003400800C200031
:1092100001002000804C8800914C880066004700C7
:10922000824C8000934C8000829FBE00512B2E0008
:10923000811F780042DC0700E68757006600470080
:1092400041F80700810037000040EB007EF6070080
:10925000E6004700802C2E00801F78000100780077
:1092600037DC07008F87E9006600470036F8070003
:1092700000C4B30074F6070050002000A7FB0700ED
:1092800080007800500020000088B900024D800066
:1092900000004100004D8800A009E20002003D00EE
:1092A0000000EB00004D8800014D800040062000CA
:1092B000808F50000200340040062000004D8800DE
:1092C00066004700A009F800912D2E00811F78004C
:1092D0001BDC0700E4875700660047001AF8070008
:1092E0005A0037000040EB0057F60700E3EC070098
:1092F000A02E2E0014F8070000C4B30052F6070099
:109300007CFB0700CF80DE00A24C8000B34C8000C5
:109310000201400083814800A24C8800B34C8800C1
:10932000E6004700A24C8000B34C8000829FBE0044
:10933000202F2E00801F78000100780000DC07003D
:10934000E687570066004700FFF707003F00370039
:109350000040EB003CF6070030302E00FAF7070023
:10936000F0EC070000C4B30037F6070050002000FF
:109370006AFB0700CF80DE00E24C8000F34C8000E7
:109380000201400083814800E24C8800F34C8800D1
:10939000E6004700E24C8000F34C8000829FBE0054
:1093A000502B2E00801F780001007800E4DB0700BE
:1093B000E687570066004700E3F707002300370001
:1093C0000040EB0020F60700C0302E00DEF707005B
:1093D00005ED070000C4B3001BF6070045FB0700BE
:1093E000CF80DE00624C8000734C800002014000A0
:1093F00083814800624C8800734C8800E600470077
:10940000624C8000734C8000829FBE00202F2E0093
:10941000801F780001007800C9DB0700E68757004D
:1094200066004700C8F70700080037000040EB005F
:1094300005F6070050312E00C3F7070000C4B30043
:1094400001F6070060322E00BFF70700630020001E
:109450009E8F11002E003A00C3C2BF000080FB00A7
:109460004400DE000080FB00610060000000E000BE
:1094700043003A00803E200060678800C3C2BF00FE
:109480000080FB004400DE000080FB006100600003
:109490000000E0003A003A00EC0CE200F7FF3A006E
:1094A000E3EA0700E4EB070087EB0700014D8000CB
:1094B000A00020000088B90080007800C0F62100DC
:1094C0004AFD07000000EB0050438800E8F5070064
:1094D00070332E009CF7070080342E00801F780028
:1094E000B6DB07008F87E900C05D200061FA070046
:1094F000C3C2BF000080FB004400DE000080FB0010
:10950000610060000000E000F9FF32002500370034
:10951000C3C2BF000080FB004400DE000080FB00EF
:10952000610060000000E00015003A00C2EB070097
:10953000014D8000C0F621002CFD07000000EB006B
:1095400050438800CAF5070040362E007EF707001A
:1095500020372E00801F780098DB07008F87E900F6
:10956000C3C2BF000080FB004400DE000080FB009F
:10957000610060000000E000F9FF320009003700E0
:10958000CFC2BF000080FB004600DE000080FB0071
:1095900061006000E10F50006DFE3A0083ED0700AE
:1095A0006BFE37000080FA00000006000600FA009B
:1095B000A0392E00801F780080DB07008F87E9002C
:1095C0000000EB00000F7800F01F20009E0F10003D
:1095D00019003C006401470000002F009E0040007D
:1095E00013002000F007200023FB0700100798005D
:1095F0001E0078006F0060000000E00006003A00E6
:109600001E007800801F7800103B2E00801F78001D
:109610006ADB0700E48757002E009000801F780067
:10962000903B2E00801F780064DB0700E487570022
:109630001E8FE800E4FF37001E009000801F7800B6
:10964000E03B2E00801F78005CDB0700E4875700BA
:109650000080FA00000006001000FA001FF9070061
:109660000000E000CD0132002CF90700204F9800E7
:109670002E4890000081FB000300200050FD2F00C9
:10968000F1FF2F000201400083814800620798002B
:109690007307980090042000010020006E019000E4
:1096A000FE019000800F5100818F5900B0013E00F3
:1096B0006E009000FE009000006001003B0137004A
:1096C000AB0137004F013700A9013700A80137006F
:1096D00069013700880137008701370086013700AC
:1096E000850137008401370083013700A00137006E
:1096F0009F013700700137009D0137009C01370042
:109700009B0137009A013700990137009801370013
:1097100097013700440037007D00370054003700C0
:10972000DE0037005000370091013700900137000C
:109730008F0137002B0037008D0137008C01370077
:109740008B0137008A013700890137008801370013
:109750008701370086013700850137009D003700FB
:109760008301370082013700810137005100370043
:109770007F0137007E013700710137007C0137001F
:109780007B0137007A013700790137007801370013
:10979000770137007601370075013700F400370094
:1097A0009A003700720137002C0137007001370032
:1097B0006F0137006E0137006D0137006C01370013
:1097C0006B013700DC00370069013700D200370039
:1097D00087003700660137006501370076003700E3
:1097E000DC003700803D2E00801F7800F3DA070090
:1097F0008F87E900F03F2E00801F7800EFDA070026
:109800008F87E90060AC2D00801F7800EBDA07003D
:109810008F87E90030412E00801F7800E7DA0700CB
:109820008F87E9005D01370090002000000F78006D
:10983000F10020009E8F100058013C001E007800AF
:109840005EF90700801F78001E017800821F7800F3
:1098500080432E00801F7800D8DA0700E687570083
:109860001E0FE800F2FF370050FF07004B013700E2
:1098700060442E00801F7800D0DA07008F87E9004F
:109880000000EB002007980012002000E11F2F00CD
:10989000F007200085FA070064004700130020004D
:1098A000E21F2F00F1072000A1FA07003FFF070089
:1098B0003A01370050462E00801F7800BFDA0700BB
:1098C0008F87E9002E489000FB4F50003301320093
:1098D00082F807000000E000FDFF32008FF807006B
:1098E000204F98002E4890000080FB00801F7800D9
:1098F00010472E00801F7800B0DA0700E487570079
:109900002E4890000080FB0068F60700EDFF37004E
:10991000D0472E00801F7800A8DA07008F87E90063
:109920000040EB00204F9800D1F407000000EB004E
:10993000000F7800F00520009E0F100008003C008A
:109940000040EB00C0F407001E00780071F507002E
:109950002003200047F907001E0FE800F5FF37003D
:1099600000C4B300B8F407002E4890000080FB004C
:10997000801F78002E4890000080FB00801F780038
:10998000E0492E00801F7800C08320006CDA0700B9
:10999000E6875700C08320006BF607002E48900032
:1099A0000040E800204F98004CF807000000E0005D
:1099B000DEFF3200F9003700A04A2E00801F780039
:1099C0007EDA07008F87E9001000200070438800CE
:1099D000F2003700104B2E00801F780077DA070066
:1099E0008F87E9000000EB0070438800EB00370030
:1099F000A008F8007608F800C04B2E00801F780001
:109A00006EDA0700E6875700E40037002609F80001
:109A1000604D2E00801F780068DA0700E487570049
:109A20002208F800404F2E00801F780063DA0700FC
:109A3000E4875700104180000000D000A39220006E
:109A40000300400010007800801F780040502E0076
:109A5000801F780059DA0700E48757003008F800C3
:109A600080522E00801F780054DA0700E4875700E8
:109A70003208F800A0532E00801F78004FDA07004C
:109A8000E48757003408F800A0542E00801F7800A7
:109A90004ADA0700E4875700C000370074F4070073
:109AA0000040EB00204F98002E489000FB4F5000E4
:109AB000BA00320009F807000000E0000900320097
:109AC00016F80700204F98002E489000E705070081
:109AD0000040EB005CF407002E4890000080FB0083
:109AE000F2F50700FC0507000000E000EEFF320081
:109AF00009060700204F98002E489000E8F707005D
:109B000000C4B30050F407002E4890000080FB0012
:109B1000E6F50700E4FF3700404C8000514C800020
:109B2000809FBE0090552E00801F780023DA07002A
:109B3000E68757009900370014FB0700801F780064
:109B4000F0562E00801F78001CDA0700E4875700CB
:109B50009200370030582E00801F780017DA070077
:109B60008F87E90010502500C6FC07008B003700E6
:109B7000C0582E00801F780010DA07008F87E90098
:109B80003E0090000000E800300798003E00900082
:109B9000BCFC0700A0002000B6F80700CFF70700C4
:109BA0000000E000F6FF32007C00370060418000DA
:109BB000219A2000010040001048E8006041800028
:109BC000229A20008200400060418000239A2000F9
:109BD0000300400010407800E348600060418000CE
:109BE000219A2000010040001080FB00801F7800B7
:109BF000A0592E00801F7800F0D90700E487570095
:109C00006600370060418000229A20000200400078
:109C10001048E90060418000239A20008300400042
:109C200060418000229A200002004000104078002D
:109C3000E348600060418000239A20000300400058
:109C40001080FB00801F7800A0592E00801F780034
:109C5000DAD90700E487570050003700B409F8004C
:109C60002C08F800105B2E00801F7800D3D9070065
:109C7000E6875700490037000A08E20007003A006B
:109C8000E05D2E00801F7800CCD907008F87E900A7
:109C9000100020005040880040003700105F2E0068
:109CA000801F7800C5D907008F87E9000000EB000E
:109CB00050408800390037000E08E20007003A00E3
:109CC00050602E00801F7800BCD907008F87E90004
:109CD000100020007040880030003700F0612E0036
:109CE000801F7800B5D907008F87E9000000EB00DE
:109CF00070408800290037002E4890000080FB004B
:109D00006F0060000000E9006040880082AD2D0017
:109D100061408000400020000008B80000004100C1
:109D20001001BE00829FBE000C08F800A0632E0048
:109D3000801F7800A1D90700E88757001700370077
:109D400070652E00801F78009CD907008F87E9007E
:109D50000000EB00000F78002E0090001E0178003C
:109D6000110009000200D800200798000B003700FE
:109D70002E4890000080FB00801F780050662E0067
:109D8000801F78008DD90700E487570020672E00D8
:109D9000801F780089D907008F87E9000080FA00CA
:109DA000000006000C00FA00881F780000B02600B2
:109DB00051542F00424C8000534C8000001F410042
:109DC000019749001E00BE00829523000201B800E1
:109DD000000278008402D0000302780005024200ED
:109DE000859523000588B9000002420084017800AF
:109DF00022079800330798004F98DE00CF80DE00DE
:109E000040079800500798002E009000BE00900078
:109E10004E019000DE019000840020008381D1007B
:109E20000281D3008180D3000080D3000402E900C6
:109E3000FAFF3A002007980031079800420798007F
:109E400053079800E8CE200014EE2D0055C62D00D3
:109E500076012000070020002E009000BE00900038
:109E60004E019000DE0190000000520081805A00F7
:109E700002015B0083815B00009CBE000294BE0077
:109E80004F0478000080FA00000006000C00FA0081
:109E90000040EB0004EDB70000CDBF000080FB00E8
:109EA0004400DE000080FB0001002000008FBE00A7
:109EB0001E00BE00A20020000203B8000001EB005B
:109EC0000282B9000701780004014100A3002000CC
:109ED0000388B900000141008203780000CDBF0073
:109EE0000080FB00010020006F0060008000EB009C
:109EF000001F430001974B001E00BE00A20020007F
:109F00000203B8000001EB000282B90007017800EB
:109F100004014100A30020000388B90000014100B2
:109F20008203780001CDBF000080FB004400DE000A
:109F30000080FB0001002000001F430001974B0040
:109F40001E00BE00A20020000203B8000001EB00CA
:109F50000282B9000701780004014100A30020003B
:109F60000388B900000141008203780001CDBF00E1
:109F70000080FB00010020006F0060008000EB000B
:109F8000001F430001974B001E00BE00A2002000EE
:109F90000203B8000001EB000282B900070178005B
:109FA00004014100A30020000388B9000001410022
:109FB0008203780002CDBF000080FB004400DE0079
:109FC0000080FB0001002000001F430001974B00B0
:109FD0001E00BE00A20020000203B8000001EB003A
:109FE0000282B9000701780004014100A3002000AB
:109FF0000388B900000141008203780002CDBF0050
:10A000000080FB00010020006F0060008000EB007A
:10A01000001F430001974B001E00BE00A20020005D
:10A020000203B8000001EB000282B90007017800CA
:10A0300004014100A30020000388B9000001410091
:10A040008203780003CDBF000080FB004400DE00E7
:10A050000080FB0001002000001F430001974B001F
:10A060001E00BE00A20020000203B8000001EB00A9
:10A070000282B9000701780004014100A30020001A
:10A080000388B900000141008203780003CDBF00BE
:10A090000080FB00010020006F0060008000EB00EA
:10A0A000001F430001974B001E00BE00A2002000CD
:10A0B0000202B8000001EB000283B900050178003C
:10A0C00006014100A30020000388B90000014100FF
:10A0D00082027800048FBE005000200001002000A2
:10A0E0001E0F40005E97480000A02500212620009A
:10A0F000BE0F1000AE8F18000300360000A0250030
:10A1000021262000008FBE001E00BE000001EB00D3
:10A110008001EB00E4CE20005403BE004402BE00E8
:10A12000C8E307002007980031079800420798000D
:10A130005307980011418000400020000008B8003B
:10A14000628A2000020240002E009000BE009000B3
:10A150004E019000DE019000F50120008381D100C6
:10A160000281D3008180D3000080D3008502E90002
:10A17000FAFF3A00008ABE000080FA0000000600E4
:10A180000200FA000000EB00000F78004000200001
:10A190009E0F100006003C0080CF20009E00400073
:10A1A0000040EB00804878001E0FE800F7FF370002
:10A1B0000080FA00000006000200FA000000EB0038
:10A1C000000F7800400020009E0F100006003C00A9
:10A1D00081CF20001E8040001040780030F607003C
:10A1E0001E0FE800F7FF37000080FA0000000600AD
:10A1F0001400FA00889FBE00044DE2000400320003
:10A2000050678000E10F400001003A001FFF070087
:10A21000EA0CE20005003A000000EB00F06788005D
:10A22000D7FF07000080EB00506788002BF607007F
:10A230000000E000C4013200800C2000506788005C
:10A24000FE0CE20002003D000000EB00F067880019
:10A25000F0678000E40F500002003400400020004E
:10A26000F0678800F067800081CF20000104400083
:10A270002AF60700004C7800F06780000000E80034
:10A28000F0678800F0678000E40F5000AE013400F2
:10A290000000EB00F0678800FCCCBF000080FB00F2
:10A2A000100F98001E099000E80F51009501320030
:10A2B0001E0A9000E80F520014003C001E08900097
:10A2C000E20F5000530132009E089000E28F5000D0
:10A2D00007003C001E0990000200E00091013200DE
:10A2E0001E0A9000E10F520076013200290037006B
:10A2F0001E089000E30F5000280032009E089000D6
:10A30000E78F500063013200220037002008200050
:10A310001E099000800F51004801320020082000E3
:10A320001E0A9000800F520009003C000008200027
:10A330009E089000808F50007F013200100820009E
:10A340001E099000800F51004701320011003700B4
:10A35000700E20001E0A9000800F5200FA0032009A
:10A36000700E20009E089000808F500005003C0079
:10A37000800820001E099000800F51006501320006
:10A3800004003700700F20001E0A9000800F52005A
:10A39000FB0032007AFF07006B01370078FF0700EF
:10A3A000D0408000E14080004F8ADE00CFA2DE0076
:10A3B000D0408000E14080000401780084017800F2
:10A3C000444C8000554C80004FACDE00CFC4DE0012
:10A3D000444C8000554C80000803780088037800C6
:10A3E00018E307004007980051079800620798009B
:10A3F000730798004E009000DE0090006E01900000
:10A40000FE019000140220008381D1000281D3005C
:10A410008180D3000080D3000402E900FAFF3A00F3
:10A4200020079800310798000040EB00F8ECB700D7
:10A43000F8CCBF004404DD002E009000BE00900068
:10A44000026829008309200023E30700004044003C
:10A45000F8ECB7002E009000BE00900002682900C2
:10A46000830920001CE30700026829000202B800EB
:10A47000820920000283B90005017800060141002D
:10A48000036829000388B9000001410082027800B6
:10A490002E009000BE0090000400500085805800FF
:10A4A00020079800310798002E009000BE00900011
:10A4B00002242400F300200007E30700F9ECB700B2
:10A4C0002E009000BE00900002242400F300200023
:10A4D00001E30700022424000202B800F200200079
:10A4E0000283B9000501780006014100032424001D
:10A4F0000388B90000014100820278002E0090001C
:10A50000BE0090000400500085805800200798008D
:10A5100031079800F9CCBF004404DD002E00900004
:10A52000BE009000026A280013002000EAE2070043
:10A5300000404400F9ECB7002E009000BE009000EF
:10A54000026A280013002000E3E20700026A2800E4
:10A550000202B800120020000283B9000501780051
:10A5600006014100036A28000388B9000001410088
:10A57000820278002E009000BE009000040050007F
:10A580008580580020079800310798002E00900021
:10A59000BE0090000271220003002000CEE20700FE
:10A5A000FAECB7002E009000BE009000027122006D
:10A5B00003002000C8E20700027122000202B80076
:10A5C0000001EB000283B90005017800060141009B
:10A5D000037122000388B900000141008202780063
:10A5E0002E009000BE0090000400500085805800AE
:10A5F0002007980031079800FACCBF004404DD0022
:10A600002E009000BE009000823E2000030020003B
:10A61000B1E2070000404400FAECB7002E009000C1
:10A62000BE009000823E200003002000AAE2070046
:10A63000823E20000202B8000001EB000283B90054
:10A640000501780006014100833E20000388B9001F
:10A6500000014100820278002E009000BE009000B0
:10A6600004005000858058002007980031079800AA
:10A670002E009000BE009000420620000300200043
:10A6800095E20700FBECB7002E009000BE009000A2
:10A6900042062000030020008FE20700420620004F
:10A6A0000202B8000001EB000283B9000501780046
:10A6B00006014100430620000388B9000001410063
:10A6C000820278002E009000BE009000040050002E
:10A6D000858058002007980031079800FBCCBF0008
:10A6E0004404DD002E009000BE009000A200200077
:10A6F0000300200078E2070000404400FBECB700B4
:10A70000104180000000D000A19220000100400014
:10A7100022002000900F110007003C001041800033
:10A720000000D000A49220000400400010407800F7
:10A73000FCECB700020037000040EB00FCECB70077
:10A740009DFE0700800037008DFE0700B0438000AB
:10A7500032002000110009000200D80000579800C4
:10A760000E509000EF4F500002003600F0C0B300D2
:10A77000005798000E509000C9F40700720037008F
:10A780007FFE0700F0448000320020001100090025
:10A790000200D800100798001E009000EF0F500034
:10A7A00002003400F0002000100798002E409000B6
:10A7B000FCECB7003408E20005003A0000C8B30022
:10A7C000C1CF20009140780000C06000FCECB700D1
:10A7D0009A08E20003003200FCCCBF000044B20043
:10A7E000FCECB70030498000E20F500006003A0050
:10A7F00040498000E20F500003003A00FCCCBF004B
:10A800000042B200FCECB700FCCCBF00A4F407008F
:10A810004D00370031498000B16788004049800011
:10A82000E20F500002003A0020002000304988006A
:10A8300020C0B3009AF4070043003700B0678000DF
:10A84000E10F500003003C00B267800032498800ED
:10A85000020037000000EB003049880020C8B30038
:10A860008FF407003800370040498000E20F5000A5
:10A8700035003A002609E200030032000000EB0038
:10A88000304988003000370010002000304988002F
:10A890002D00370080CF200024C0B300904F12005D
:10A8A00029003E00104180000000D000A29220004C
:10A8B00082004000F8CCBF000080FB0080087800D8
:10A8C000210037000000EB00000F7800440020005A
:10A8D0009E0F12001C003C0000D020009E00400093
:10A8E00082CF20001E0041009048780084CF2000D5
:10A8F0009E0042000040EB00804878001E0FE800F8
:10A90000F2FF3700CAE2A80080C0B30064F4070079
:10A910000D003700CAE2A90080C8B30060F4070048
:10A920000900370010002000604388000040EB0061
:10A930005BF40700040037000000EB006043880070
:10A9400000C8B30056F407004F04BE000080FA00B0
:10A95000000006000200FA000000EB00000F780083
:10A96000F04B8000E20F500005003A005BF4070056
:10A970000000E0000200320010002000000F78000C
:10A98000550207000000E000020032001000200025
:10A99000000F78001E0078000080FA00000006001A
:10A9A0000000FA00E922A800E8C2A800E902A90014
:10A9B0000080FA00000006000600FA00000F780090
:10A9C0000000EB00100798001E009000EF0F5000F1
:10A9D0001D003C00E8C2A9009E0078006180600074
:10A9E0000000E00002003200E902A8000100370088
:10A9F000E902A9001E0078000000D100000F7800D5
:10AA00002E0090000000D10020079800E6C2BF0091
:10AA10000080FB004700DE000080FB000000E0003B
:10AA2000040032002E009000010028000100700098
:10AA300020079800E8C2A8001E0090000000E8006F
:10AA400010079800E0FF37002E0090000080FA0009
:10AA5000000006000400FA00000F7800E922A900B7
:10AA60001E007800D4FF070010079800E922A80014
:10AA7000E902A9001E0090000080FA000000060014
:10AA80000600FA00000F780011079800E922A900DB
:10AA90001E007800C8FF07001E009000C6FF0700D8
:10AAA00020079800E922A800E902A9002E009000E2
:10AAB0000080FA00000006000A00FA00000F78008B
:10AAC0001107980022079800E922A9001E007800CB
:10AAD000B9FF0700300798001E009000B6FF07007E
:10AAE000300798002E009000B3FF07003007980051
:10AAF000E902A9000000EB00400798004E0090001A
:10AB0000E70F50000A003C00E8C2A9000000000066
:10AB100000000000E8C2A8000000000000000000E3
:10AB20004E0090000000E80040079800F3FF370057
:10AB3000E922A800E902A9003E0090000080FA0086
:10AB4000000006000200FA00E9C2A80094FF070016
:10AB500010002000BFFF0700D10020005086280011
:10AB6000C7FF07008000EB0090002000C4FF070033
:10AB700080007800F00F2000008F60000000EB00E4
:10AB8000D0418800000E20009E0F100009003A00FE
:10AB9000D100200050862800B9FF0700006B2E006E
:10ABA000801F780005D607008F87E900100020007D
:10ABB000D04188000080FA00000006000200FA0080
:10ABC000000F780082682E009E0078004000200070
:10ABD0000008B8000000410010007800806988007B
:10ABE00082682E009E007800400020000008B80017
:10ABF000000041000080E8001000780090698800A3
:10AC00000080FA00000006000400FA00000F78003F
:10AC1000110798000000EB00B041880014F0070015
:10AC20001E0090000000E00008003A001E007800BE
:10AC3000801F7800406E2E00801F7800C0832000A7
:10AC4000BFD50700E48757000A003700CBF607009E
:10AC5000401F2000104588001E007800801F7800EB
:10AC6000406F2E00801F7800C0832000B4D50700FD
:10AC7000E4875700C0832000B3F10700D100200013
:10AC800050862C007EFF07001E007800CBFF0700D7
:10AC9000400020006FFF07009269800081698000FA
:10ACA0000009200084FF0700E7C2BF000080FB000E
:10ACB0004400DE000080FB00610060000000E00056
:10ACC000180032001E0090000000E0000600320074
:10ACD00080C0B300DCEF0700D000200037F407008D
:10ACE000C043880087E6070000C4B300D6EF070022
:10ACF0003608F800E06F2E00801F7800C083200027
:10AD00008FD50700E4875700C08320008EF107002D
:10AD100010FF07000000E000E3FF320020012000E8
:10AD20004CFF0700D10020005086280054FF070088
:10AD30000080FA00000006000400FA00000F78000E
:10AD4000110798000000EB00B0418800C8EF070031
:10AD50001E0090000000E0000B003A001E0078008A
:10AD6000801F7800E0702E00801F7800C0832000D4
:10AD700073D50700E4875700D100200050062C004F
:10AD80003FFF07000D0037007CF60700401F200042
:10AD9000104588001E007800801F780010722E0079
:10ADA000801F7800C083200065D50700E487570026
:10ADB000D10020005086280031FF0700C08320000A
:10ADC00061F1070000C4B3009FEF07001E00780088
:10ADD0007AFF0700400020001EFF070092698000F4
:10ADE000816980002009200033FF0700E7C2BF000F
:10ADF0000080FB004400DE000080FB00610060007A
:10AE00000000E000F9FF3A004000200011FF0700B9
:10AE100092698000816980001009200026FF0700E8
:10AE2000E7C2BF000080FB004400DE000080FB00A2
:10AE3000610060000000E000150032001E0090007C
:10AE40000000E0000300320080C0B3007EEF070086
:10AE50002CE6070000C4B3007BEF07003608F800BB
:10AE6000E06F2E00801F7800C083200034D50700DB
:10AE7000E4875700C083200033F10700B5FE0700C8
:10AE80000000E000E6FF320020012000F1FE070094
:10AE900040002000EFFE0700D1002000508628006F
:10AEA000F7FE07000080FA00000006000800FA0024
:10AEB0000AF307000000E000AE00320017F30700BD
:10AEC000204798003A08E20002003A000040EB00F8
:10AED000204798002E4090000080FB00300798002B
:10AEE000D0042000BE009000808F50002A00320065
:10AEF000D0042000BE009000808F500011003C0064
:10AF000090032000BE009000808F500008003C009D
:10AF100000032000BE009000808F500043003D00E1
:10AF20003E0090000000E000890032008D003700F4
:10AF300050042000BE009000808F50002C00320092
:10AF40008800370020052000BE009000808F500050
:10AF50001100320020052000BE009000808F5000BC
:10AF600005003C0000052000BE009000808F5000CE
:10AF7000090032007B00370030052000BE00900041
:10AF8000808F50001000320040052000BE0090006D
:10AF9000808F500073003A002E40900036EDB700CD
:10AFA000014D8000108F210090F60700C0722E0026
:10AFB000801F780001D507008F87E9002E409000A0
:10AFC000B7F207006B003700F0732E00801F780087
:10AFD000FAD407008F87E900200120009DFE0700BA
:10AFE000014D8000108F210080F6070061003700BE
:10AFF000A0752E00801F7800F0D407008F87E9002D
:10B00000014D8000A00020000088B9008000780079
:10B01000108F210075F60700300520008DFE070017
:10B020000040EB0036EDB700520037002E40900094
:10B030000080FB0001FD2F0001004000A069880096
:10B04000340DF80030772E00801F7800DBD4070025
:10B05000E4875700A0698000D8FE070036CDBF0006
:10B060000080FB002007980000052000AE00900043
:10B07000808F50001200320000052000AE009000CA
:10B08000808F500005003C00D0042000AE009000EE
:10B09000808F500026003200360037002005200047
:10B0A000AE009000808F5000190032004005200053
:10B0B000AE009000808F5000090032002D00370054
:10B0C000E0772E00801F7800BCD407008F87E9004E
:10B0D0008000EB00A0698000CBFE07002500370050
:10B0E00000792E00801F7800B4D407008F87E90014
:10B0F000E9E2A800CAE2A80011002000A0698000CF
:10B10000C1FE0700CAE2A900E9E2A9001900370060
:10B1100090792E00801F7800A8D407008F87E9005F
:10B1200011002000A069800003FF07001100370014
:10B13000107A2E00801F7800A0D407008F87E900C6
:10B140008000EB00A0698000FBFE070009003700CB
:10B15000707B2E00801F780098D407008F87E9004D
:10B1600004003700B07D2E00801F780093D40700C4
:10B170008F87E9000080FA0000000600809FBE0073
:10B180000200FA00E0108000004F780040CDBF00C0
:10B190000080FB008000E800C2CABF000080FB0006
:10B1A000808F50000800320040CDBF000080FB00BF
:10B1B00031AC2000010040001E48780040CDBF00A7
:10B1C0000040E80040EDB70018C2BF000080FB005F
:10B1D0000000D1000080FB0061006000E10F500022
:10B1E00001003A001822A9008700A9000080FA0097
:10B1F0004F00BE00004006000000FA00E07D2E0077
:10B2000030009000F01088000000EB00B0108800C3
:10B2100000402000C01088008700A9008F00A8000F
:10B2200017E2A8001942A8000080FA0000000600FA
:10B230000200FA00000F7800700020009E0F10003E
:10B240000200340070002000000F7800E17D2E0025
:10B250001E0078000000D0000100400010007800BF
:10B26000F01088000080FA00000006000200FA00DA
:10B27000004F780019C2BF000080FB000000D10021
:10B280000080FB0061006000E10F5000F9FF320018
:10B290001E00FB00F10F200001006000D0108800AC
:10B2A0000080FA00000006000200FA00000F78009B
:10B2B0001E0078001004E000050032001E00780037
:10B2C00010407800E9FF07001E0FE800F8FF370084
:10B2D0000080FA00000006000200FA0001D42000FD
:10B2E00091407800C2CABF0000C05000004FE90082
:10B2F0001E80FB000080FA00000006000000FA003B
:10B300000040EB00C2EAB70010C0B30040EDB70048
:10B310000080FA00000006000000FA0000000000B3
:10B32000C2CABF000080FB008000E80040CDBF0023
:10B330000080FB00808F5000F9FF3200C2CABF00BE
:10B340000040E800C2EAB7000080FB0031AC2000FA
:10B35000010040001080FB000080FA0000000600A1
:10B360000200FA00ECFF0700004F78001E40780052
:10B37000BEFF07001E80FB000080FA0000000600F0
:10B380000800FA00D4FF07000000E0007D00320052
:10B39000E1FF0700204798003A08E20079003200F8
:10B3A0002E4090000080FB0030079800D004200061
:10B3B000BE009000808F500026003200D004200094
:10B3C000BE009000808F50000D003C000003200064
:10B3D000BE009000808F50006A003500900320006E
:10B3E000BE009000808F50003300340050042000D5
:10B3F000BE009000808F50002400320061003700B2
:10B4000020052000BE009000808F50001100320007
:10B4100020052000BE009000808F500005003C00F9
:10B4200000052000BE009000808F5000090032000F
:10B430005400370030052000BE009000808F50007F
:10B440000A00320040052000BE009000808F5000AE
:10B450004C003A002E4090003AEDB700014D8000BC
:10B46000108F210061F50700460037002001200001
:10B4700078FD0700014D8000108F21005BF507006B
:10B480000040EB003AEDB7003E003700014D800070
:10B49000A00020000088B90080007800108F2100F3
:10B4A00052F50700300520006AFD07000040EB0060
:10B4B0003AEDB700330037002E4090000080FB00CB
:10B4C00001FD2F0001004000C0698800C0698000B4
:10B4D000BAFD07003ACDBF000080FB0020079800AE
:10B4E00000052000AE009000808F50001200320056
:10B4F00000052000AE009000808F500005003C0049
:10B50000D0042000AE009000808F50001A0032005E
:10B510001C00370020052000AE009000808F5000F6
:10B520001100320040052000AE009000808F5000D6
:10B5300005003200130037008000EB00C069800076
:10B54000B1FD07000F003700E9E2A800CAE2A80039
:10B5500011002000C0698000ABFD0700CAE2A9000D
:10B56000E9E2A9000700370011002000C06980004F
:10B57000F1FD0700030037008000EB00C069800088
:10B58000EDFD07000080FA000000060020760000B4
:10B59000312E00003033000000310000312E000059
:10B5A000303300002E320000303000003800000040
:10B5B0000100000000000000640000000000000026
:10B5C000E803000000000000102700000000000059
:10B5D000A086000001000000404200000F000000B3
:10B5E0003000000000000000DD010000000000004D
:10B5F000A4120000000000006ABA00000000000071
:10B6000023480000070000005AD100004800000055
:10B61000610B0000B6000000C11600006C010000C4
:10B62000832D0000D8020000065B0000B00500007A
:10B630000BB60000600B0000176C0000C116000084
:10B64000ABAA0000AA2A0000610B0000B6000000AF
:10B65000C11600006C010000832D0000D80200001C
:10B66000065B0000B00500000BB60000600B000098
:10B67000176C0000C11600002222000022220000E8
:10B68000ABAA0000AA2A0000B66000000B3600003A
:10B69000C11600006C4100004A9F0000F449000000
:10B6A0000000000000010000000200000003000094
:10B6B0000004000000050000000600000006000075
:10B6C000000700000007000000070000000700005E
:10B6D0003132000030300000202000000000000067
:10B6E0003234000030300000202000000000000054
:10B6F000343800003030000020200000000000003E
:10B70000393600003030000020200000000000002A
:10B71000313900003230000030200000000000000D
:10B7200033380000343000003020000000000000FA
:10B7300035370000363000003020000000000000E7
:10B7400031310000353200003030000020000000B0
:10B750003A000000210000001200000096000000E6
:10B760003A000000210000000A0D0000576F0000A1
:10B7700072640000732000003D200000256400007A
:10B780002C200000537500006365000073730000F7
:10B79000203D000020250000642C00002043000014
:10B7A00068650000636B0000737500006D20000089
:10B7B0003D20000025580000000A00000D57000041
:10B7C0006F72000064730000203D0000202500001F
:10B7D000642C0000205300007563000063650000C6
:10B7E00073730000203D000020250000642C000041
:10B7F0002043000068650000636B00007375000063
:10B800006D2000003D200000255800000050000081
:10B81000575200000050000057520000202D000039
:10B820002E2D000057000000494400000041000098
:10B8300000490000442000002D2E00002D2D0000A6
:10B840004100000052460000205000006F770000C9
:10B8500065720000203D0000200000002064000010
:10B860004200000050770000722000004F460000A8
:10B870004620000061660000746500007220000030
:10B88000256900002020000000560000464F0000FF
:10B89000206C00006F6300006B200000202000007F
:10B8A00020200000204F00004E00000056460000FF
:10B8B0004F2000006C6F0000636B00002020000030
:10B8C00020200000204F000046460000000A000033
:10B8D0000D550000736500007220000073650000C4
:10B8E00074740000696E000067730000207300002C
:10B8F0006176000065640000207400006F20000085
:10B9000045450000505200004F4D00002C20000023
:10B91000506F000077650000722000006F66000025
:10B92000660A00000D000000525300003233000090
:10B9300032200000546500007374000020200000D5
:10B940002020000020200000005700006169000056
:10B95000746900006E6700002064000061740000DC
:10B96000612E00002E2E00002E0000005258000014
:10B9700020640000617400006120000020000000CD
:10B980002020000030780000004A0000554D0000E3
:10B99000412D0000545200005832000020000000E9
:10B9A000202000004F480000324E00004C540000A0
:10B9B000204F0000483700005356000020200000B0
:10B9C000000A00000D0A00000D4A0000554D00005D
:10B9D000412D000054520000583200002046000063
:10B9E000697200006D770000617200006520000040
:10B9F000002C000020420000756900006C6400000B
:10BA0000200000000A0D0000436F00007079000064
:10BA10007269000067680000742000004A75000029
:10BA200068610000204E0000696900006E69000036
:10BA30006B6F0000736B0000692C0000204F00004A
:10BA4000483200004E4C0000540A00000D0A00006D
:10BA50000D0000005379000073740000656D000054
:10BA6000204300006C6F0000636B0000203D00006D
:10BA700020250000692000006B4800007A0A0000C1
:10BA80000D0000004A5500004D4100002D540000FB
:10BA9000525800003220000055410000525400006E
:10BAA0003220000066690000786500006420000014
:10BAB000393600003030000020620000640A0000C7
:10BAC0000D000000506F000077650000722000003C
:10BAD0004F4E0000005300006572000076690000C0
:10BAE00063650000204D00006F64000065200000C9
:10BAF0002020000020000000507500007368000046
:10BB00002044000049530000504C000041590000FF
:10BB1000206E000078740000005000007573000073
:10BB2000682000004641000053540000203D000002
:10BB30002053000061760000650000000A0D00003F
:10BB400045450000505200004F4D000020630000AA
:10BB500068650000636B0000737500006D73000082
:10BB60002C200000436100006C2000003D200000FC
:10BB7000255800002C2000004465000066200000CD
:10BB800043730000203D000020250000582C0000D9
:10BB90002046000061630000746F000072790000AD
:10BBA0002064000065660000617500006C74000090
:10BBB00020720000657300006574000073200000AF
:10BBC0003D20000025640000000A00000D45000033
:10BBD00045500000524F00004D20000063680000F7
:10BBE000656300006B730000756D00002065000048
:10BBF000727200006F7200002C200000726500005D
:10BC00006C6F00006164000020660000616300004A
:10BC1000746F000072790000206400006566000007
:10BC2000617500006C740000730000005075000026
:10BC30007368000020530000455400002066000097
:10BC40006F7200002020000020200000006600002D
:10BC500061630000746F00007279000020640000CE
:10BC600065660000617500006C74000073000000E0
:10BC70000A0D0000536500007420000055410000CB
:10BC800052540000312000007573000065720000FE
:10BC900020620000617500006420000072610000F5
:10BCA00074650000207400006F2000002325000050
:10BCB000692C000020200000257300006264000051
:10BCC0000A0D0000000A00000D530000657400001A
:10BCD0002055000041520000542000007573000000
:10BCE00065720000206200006175000064200000A1
:10BCF0007261000074650000207400006F20000075
:10BD000023250000692C000020200000257300007E
:10BD1000626400000A0D000000560000464F00005B
:10BD2000412000003D3E000020560000464F00002C
:10BD3000422000006F6B0000200000004C53000008
:10BD40004200000055530000420000002043000064
:10BD500057000000547500006E65000000200000D0
:10BD60002054000058000000204E00004152000006
:10BD7000002000004D490000440000002057000052
:10BD8000494400000053000057520000002000000A
:10BD90004E2F0000412000000053000057520000C9
:10BDA000202D00002E2D00002D000000200000009E
:10BDB00056000000232500006C5800000020000001
:10BDC0005200000020530000706C0000740000005E
:10BDD00020560000464F00000020000053000000E5
:10BDE0002046000000200000560000002020000037
:10BDF000204C00006F6300006B0000002041000039
:10BE0000646A000075730000740000004147000080
:10BE1000432000003D2000004661000073740000D4
:10BE20002020000020200000202000000041000011
:10BE300047430000203D0000205300006C6F0000CD
:10BE400077200000202000002020000020000000BB
:10BE50004E410000520000004D4900004400000027
:10BE60005749000044000000204C000050460000EC
:10BE700020200000002500006C6900002048000020
:10BE80007A200000200000004E420000206F0000D9
:10BE900070740000696F00006E2000003D200000FB
:10BEA0004F4E000020200000004E00004220000005
:10BEB0006F700000746900006F6E0000203D00008C
:10BEC000204F000046460000200000005370000094
:10BED0006565000063680000507200006F63000039
:10BEE000203D0000204F00004E20000000530000C5
:10BEF000706500006563000068500000726F00000C
:10BF0000632000003D2000004F4600004600000076
:10BF100041460000206900006E2000003D20000026
:10BF20004C6900006E650000202000002020000009
:10BF30000041000046200000696E0000203D000026
:10BF4000204D000069630000202000002020000038
:10BF5000200000004B6500007965000072200000A1
:10BF60003D200000004400006F74000020700000BD
:10BF7000726900002E000000496100006D6200003F
:10BF8000696300002041000000490000616D00006D
:10BF9000626900006320000042000000537400004A
:10BFA00072610000696700006874000000430000CF
:10BFB00057200000706900007463000068200000D2
:10BFC00025690000204800007A20000020000000C1
:10BFD00043570000207000006F740000203D0000F7
:10BFE0002053000071750000656C0000636800005C
:10BFF0000043000057200000706F00007420000014
:10C000003D2000004357000073700000656500008C
:10C01000640000004C43000044200000424C00003B
:10C02000203D0000202500006920000020200000A5
:10C030002020000020000000436F00006E7400000C
:10C040007261000073740000203D00002025000094
:10C05000692000002000000052530000323300002D
:10C06000322000003D200000004A0000554D000035
:10C070004154000052580000320000005961000095
:10C080006573000075430000415400000056000035
:10C090006F690000636500004D6500006D000000E1
:10C0A0005465000073740000202000002020000070
:10C0B0000042000061750000642000005261000031
:10C0C000746500003D250000730000005646000026
:10C0D0004F2000003D200000412F000042200000C2
:10C0E0002B200000537000006C740000005600000C
:10C0F000464F0000203D0000202500006920000080
:10C100004D6500006D200000202000002020000070
:10C11000004600002025000069200000256900007D
:10C120002057000020000000522000002569000078
:10C13000202500006920000057200000000A0000B0
:10C140000D540000525800005F320000206D0000C6
:10C150006F640000652000006E6F00007420000016
:10C160007965000074200000696D0000706C0000AB
:10C17000656D0000656E000074650000640A0000D3
:10C180000D0000002000000000010000010200007E
:10C190002003000003040000040200000606000063
:10C1A00006060000050700000707000086010000E2
:10C1B000C200000061000000300000001700000015
:10C1C0000B00000007000000030000000A0D000043
:10C1D0004F750000745F0000697800006420000063
:10C1E000256900002C200000496E00005F690000F6
:10C1F000647800002025000069200000200A00006B
:10C200000D0000000A0D00005452000041500000D3
:10C210003A2000004F730000636900006C61000069
:10C22000746F00007220000045720000726F000001
:10C23000720A00000D0000004F530000434300004D
:10C240004F4E00002030000078250000580A000002
:10C250000D0000000A0D0000545200004150000083
:10C260003A20000041640000647200006573000021
:10C270007320000045720000726F0000720A000017
:10C280000D0000005730000020300000782500002D
:10C29000580A00000D000000573100002030000057
:10C2A00078250000580A00000D00000057320000F9
:10C2B0002030000078250000580A00000D00000022
:10C2C000573300002030000078250000580A000095
:10C2D0000D000000573400002030000078250000D9
:10C2E000580A00000D000000573500002030000003
:10C2F00078250000580A00000D00000057360000A5
:10C300002030000078250000580A00000D000000D1
:10C31000573700002030000078250000580A000040
:10C320000D00000057380000203000007825000084
:10C33000580A00000D0000005739000020300000AE
:10C3400078250000580A00000D0000005731000059
:10C350003020000030780000255800000A0D000051
:10C360000057000031310000203000007825000027
:10C37000580A00000D000000573100003220000074
:10C3800030780000255800000A0D0000005700001A
:10C39000313300002030000078250000580A0000EA
:10C3A0000D000000573100003420000030780000FC
:10C3B000255800000A0D000000570000313500002C
:10C3C0002030000078250000580A00000D00000011
:10C3D0000A0D000054520000415000003A200000B5
:10C3E00053740000616300006B2000004572000080
:10C3F000726F0000720A00000D0000000A0D0000BC
:10C4000054520000415000003A2000004D610000ED
:10C410007468000020450000727200006F72000016
:10C420000A0D0000000A00000D53000070750000A6
:10C43000726900006F75000073200000496E0000F3
:10C4400074650000727200007570000074200000B6
:10C4500045720000726F0000720A00000D000000BB
:10C46000202000002020000045720000726F0000B4
:10C470007220000021200000202000002020000069
:10C48000000000000A0D00005365000072760000F5
:10C490006963000065200000262000006361000041
:10C4A0006C6900006272000061740000696F000036
:10C4B0006E2000006D6F000064650000000A00003F
:10C4C0000D460000554E0000432000003D200000B6
:10C4D00070610000726100006D650000746500000D
:10C4E00072200000736500006C650000637400003A
:10C4F0002C20000053450000542000003D20000087
:10C5000073610000766500002026000020650000B1
:10C51000786900007400000053650000742000007A
:10C5200052650000662000004F7300006320000089
:10C530004672000065710000004F00007363000048
:10C54000202500006C690000204800007A000000EF
:10C5500053750000707000006C790000202000000E
:10C56000005600002020000000430000616C000025
:10C57000206D0000756C0000742000003D2000005C
:10C58000256C000069200000202000002000000031
:10C590004265000065700000206C0000656E0000C0
:10C5A0002C200000303D00004F46000046200000D7
:10C5B0000042000065650000702000003D20000082
:10C5C00025690000206D000073200000202000007D
:10C5D00020000000532D00006D6500007465000010
:10C5E00072000000436100006C2000006D750000C7
:10C5F0006C740000203D0000202500006C690000E4
:10C6000020200000004600006F72000077610000EB
:10C61000726400002000000052460000204100002B
:10C620006D7000002E2000000050000075730000A7
:10C63000682000004641000053540000206C0000B8
:10C640006F6E0000672000003D0000006661000082
:10C65000637400006F7200007920000064650000C0
:10C6600066610000756C00007473000000460000F5
:10C6700061630000746F0000727900002073000095
:10C680006574000075700000206F00006B000000F2
:10C690000A0D000046610000637400006F72000024
:10C6A000792000006465000066610000756C000080
:10C6B000747300002072000065730000746F000046
:10C6C0007265000064000000436100006C690000B6
:10C6D000627200002E2000005361000076650000A9
:10C6E000640000000A0D0000436100006C69000056
:10C6F0006272000061740000696F00006E2000002B
:10C700007365000074740000696E000067730000B8
:10C710002073000061760000656400002074000052
:10C720006F20000045450000505200004F4D0000B2
:10C7300000000000447500006D70000020450000FE
:10C7400045500000524F00004D200000636F000074
:10C750006E740000656E0000747300000A0D000026
:10C76000000A00000D250000352E0000345800009E
:10C770000020000025340000580000000A0D0000D1
:10C780004C610000737400002073000075630000AA
:10C790006365000073730000206300006F64000095
:10C7A000652000003D20000025580000200000000A
:10C7B0000A0D00004A5500004D4100002D540000B4
:10C7C0005258000032200000636F000070790000B2
:10C7D0007269000067680000742000004F48000084
:10C7E0003753000056200000262000004F4800006C
:10C7F000324E00004C5400000A0D0000000A0000F8
:10C800000D5300006F660000747700006172000035
:10C81000652000007665000072730000696F0000FB
:10C820006E200000002C0000206300006F700000EC
:10C83000797200006967000068740000204A0000F7
:10C8400075680000612000004E690000696E0000FC
:10C85000696B00006F7300006B690000204F0000DF
:10C86000483200004E4C0000540A00000D00000049
:10C870000A0D00004144000043200000256900002B
:10C88000203D000020250000690000004545000013
:10C89000505200004F4D00002072000065730000F0
:10C8A00065740000206300006F7500006E74000066
:10C8B00065720000206300006C650000617200007A
:10C8C000656400000A0D0000004C000043440000B5
:10C8D0002077000072690000746500000A0D0000F6
:10C8E0000063000068610000722000003D2000002D
:10C8F000257800000A0D0000004C000043440000B1
:10C900002062000061720000206700007261000078
:10C9100070680000202600002063000068610000AD
:10C9200072610000637400006572000020740000F2
:10C9300065730000740A00000D000000256300000C
:10C94000203D000020300000782500005820000025
:10C95000200000000A0D00004D7500007465000005
:10C96000000A00000D41000075640000696F0000BE
:10C97000206F00006E0000000A0D0000535F0000F1
:10C980006D65000074650000722000003D2000000D
:10C99000253100002C5000004F540000203D0000C5
:10C9A00020250000690A00000D0000000A0D0000AB
:10C9B0002065000065700000726F00006D2E0000A1
:10C9C0006465000066760000616C00002E76000051
:10C9D000666F00005F730000656C0000203D000082
:10C9E00020250000690000000A0D000020760000EC
:10C9F000666F00005F69000064780000203D000061
:10CA000020250000690000000A0D000020650000DC
:10CA100065700000726F00006D2E000064650000FC
:10CA200066760000616C00002E6D00006F640000EF
:10CA3000655B0000766600006F5F000069640000BF
:10CA4000785D0000203D0000202500006900000006
:10CA50000A0D000020630000775F000061630000A2
:10CA60007469000076650000203D0000202500006C
:10CA7000690000000A0D000020740000756E0000BF
:10CA8000655F00006F6E0000203D00002025000063
:10CA9000690000000A0D00002050000054540000FE
:10CAA0005F4900004E2000003D2000002569000085
:10CAB000000A00000D52000065660000204F0000D3
:10CAC00073630000203D0000202500006C69000019
:10CAD000204D0000487A00000A0D0000000A000006
:10CAE0000D6D000073200000636F0000756E000084
:10CAF00074650000722000003D20000025690000E0
:10CB00000A0D0000000A00000D530000504900000B
:10CB100020540000780000000A0D0000535000006F
:10CB20004920000054780000206300006F6E000070
:10CB3000740000000A0D0000504100002041000078
:10CB400074740000656E000075610000746F000071
:10CB5000722000003D2000003078000025580000C1
:10CB6000000A00000D520000462000004174000041
:10CB7000746E000020730000656C000065630000A7
:10CB80007420000069640000782000003D2000004F
:10CB9000256900002C2000004843000035390000C2
:10CBA000352000006269000074730000203D000021
:10CBB0002030000078250000580000000A0D000019
:10CBC0004444000053200000747500006E650000AE
:10CBD0002074000065730000742000004F4E0000B8
:10CBE000000A00000D4400004453000020740000BF
:10CBF000756E00006520000074650000737400000D
:10CC0000204F000066660000000A00000D4400008E
:10CC10004453000020740000756E0000696E00002F
:10CC200067200000776F000072640000206400003D
:10CC300069730000706C000061790000000A000058
:10CC40000D4E00006F7200006D6100006C2000004E
:10CC50004672000065710000756500006E6300009B
:10CC60007920000064690000737000006C610000AE
:10CC7000790000000A0D0000444400005320000029
:10CC8000747500006E6900006E670000207300007C
:10CC9000746500007020000023200000256900005A
:10CCA000203D0000202500006C690000000A000003
:10CCB0000D44000069760000206200007920000029
:10CCC0005A650000726F0000004B0000657900009B
:10CCD00020690000733A000020250000640A00006B
:10CCE0000D00000054720000793A00002056000048
:10CCF000616C000069640000206300006F6D00003B
:10CD00006D6100006E640000730A00000D000000F9
:10CD100010000000FF03000000040000AF0400004A
:10CD2000B004000007050000080500005F050000D2
:10CD300060050000B7050000B80500000F06000000
:10CD4000100600006706000068060000BF0600002D
:10CD5000C006000017070000180700008F0700003A
:10CD60000A0D000054520000582D0000322000002F
:10CD7000766F000069630000652000006D650000AB
:10CD80006D6F000072790000206F00007074000069
:10CD9000696F00006E200000666F0000756E000075
:10CDA000642000002849000053440000313700008F
:10CDB0003234000030200000636800006970000019
:10CDC000290A00000D000000504C000041590000ED
:10CDD000204D0000656D000020230000202500008C
:10CDE000692000002000000054580000204D000081
:10CDF0002025000069200000200000005469000088
:10CE00006D650000202500006920000073200000EF
:10CE100020200000202000002000000052450000DB
:10CE2000432000004D69000063200000204D0000F9
:10CE3000656D00002023000020250000692000000F
:10CE400000520000582000004D200000256900001D
:10CE500020200000000000000A0D0000566F0000B6
:10CE600069630000652000004D6500006D20000032
:10CE7000636D0000642000003D200000000A0000F7
:10CE80000D5600006F69000063650000204D000032
:10CE9000656D000020530000746F000070200000DA
:10CEA0006F7000006572000061740000696F00001F
:10CEB0006E0000000A0D0000566F0000696300005C
:10CEC000652000004D6500006D6F00007279000064
:10CED00020650000726100007365000020610000A1
:10CEE0006C6C0000000A00000D4D0000656D000034
:10CEF000203D000020250000690000000A0D000010
:10CF0000564D00002C200000706C0000617900007C
:10CF1000206D0000656D00006F7200007900000058
:10CF20000A0D0000564D00002C200000545800004F
:10CF3000000A00000D5600004D200000525800006D
:10CF4000000A00000D5600004D2C00002052000089
:10CF5000656300006F7200006420000066720000CC
:10CF60006F6D0000204D000069630000000A0000A2
:10CF70000D5600006F69000063650000204D000041
:10CF8000656D00006F720000792000006F70000076
:10CF9000746900006F6E0000206E00006F74000066
:10CFA000206900006E730000746100006C6C00006A
:10CFB00065640000003F00000000000086010000E2
:10CFC000C2000000610000003000000017000000F7
:10CFD0000B00000007000000030000003C0D0000F3
:10CFE0000200000002000000000000000008000035
:10CFF000B601000000000000B60900000C010000AE
:10D00000000000003E0D00000200000002000000D1
:10D0100001000000180D00000600000000000000E4
:10D020001E0D00000600000000000000B60C00000D
:10D030002000000000000000D60C000018000000D6
:10D0400000000000240D00000600000000000000A9
:10D05000EE0C00001800000000000000300D000081
:10D060000400000000000000340D00000400000077
:10D0700000000000C20A00000201000000000000E1
:10D08000400D00000200000002000000010000004E
:10D09000380D00000400000000000000C40B000078
:10D0A00088000000020000000100000000EA0B0000
:10D0B000EB0BEA000BEA0B00EA0BEA000BDA0B00C1
:10D0C0000000000000000000000000000000000060
:10D0D0000000000000000000000000000002080046
:10D0E000010112000C130C00120C12000C120C00A7
:10D0F000120C02000C000000000000000000000004
:10D10000000000000000000000000000000000001F
:10D1100000000200080202003A0C3B000C3A0C002E
:10D120003A0C3A000C3A0C002A0C000000000000F7
:10D1300000000000000000000000000000000000EF
:10D140000000000000000000C40BEC000B140C00F9
:10D1500000000000000000000000000000000000CF
:10D16000060D00001200000002000000202B2D0020
:10D17000233000000100020000040000080010003D
:10D18000000000007E0D000008000000020000000A
:10D19000686A6C00747A4C00000000002A0D0000E0
:10D1A0000600000002000000000000000000020075
:10D1B000420D00000200000000000000940C00007E
:10D1C000220000000200000030313200333435000C
:10D1D00036373800396162006364650066003000EC
:10D1E000313233003435360037383900414243009C
:10D1F00044454600000000004C0C000048000000C0
:10D2000002000000000000000000000024400000B8
:10D210000000000000005900400000000000000075
:10D2200088C34000000000000084D7009741000040
:10D2300080E0370079C3410043176E0005B5B500A3
:10D24000B8934600F5F93F00E9034F00384D32002E
:10D250001D30F900487782005A3CBF00737FDD0023
:10D260004F1575004C0D0000320000000200000058
:10D270004E414E00006E61006E0049004E460000B7
:10D28000696E6600003031003233340035363700C5
:10D290003839610062636400656600003031320035
:10D2A00033343500363738003941420043444500B5
:10D2B00046000000440D00000200000002000000D3
:10D2C00000000000860D00000200000002000000C7
:10D2D00030000000460D00000200000002000000C7
:10D2E00000000000480D00000200000002000000E5
:10D2F000010000004A0D00000200000000000000D4
:10D30000000000000000000000000000000000001D
:10D31000000000000000000000000000000000000D
:10D3200000000000000000000000000000000000FD
:10D3300000000000000000000000000000000000ED
:020000040002F8
